:100000000040002049510000895100008B51000040
:1000100000000000000000000000000000000000E0
:100020000000000000000000000000008D510000F2
:1000300000000000000000008F51000091510000FE
:100040009351000055390000C55500009351000040
:1000500093510000000000009351000093510000F4
:1000600093510000955800009351000093510000F7
:1000700093510000935100009351000093510000F0
:10008000935100002D5A000093510000935100003D
:1000900093510000935100009351000093510000D0
:1000A0009351000093510000000000000000000088
:1000B0000000000000000000000000000000000040
:1000C00010B5064C2378002B07D1054B002B02D02E
:1000D000044800E000BF0123237010BD4802002047
:1000E00000000000F8B70000044B10B5002B03D04F
:1000F0000349044800E000BF10BDC04600000000F6
:100100004C020020F8B70000164B002B00D1144B16
:100110009D46402292029A1A924600218B460F4633
:100120001348144A121A08F0C2FD0F4B002B00D0DE
:1001300098470E4B002B00D0984700200021040068
:100140000D000D48002802D00C4800E000BF08F068
:100150006DFD2000290005F053FA08F041FDC0466E
:100160000000080000400020000000000000000027
:1001700048020020C8250020000000000000000008
:1001800002000120104004D1042A01D9106800099E
:1001900070470020FCE710B50400FFF7F1FF0028CE
:1001A00009D001388000031D22181279002A02D0DC
:1001B00001309842F8D110BD0122096810B51142F2
:1001C00001D0002903DA102000F084F910BD491095
:1001D000062002F05DF8F9E7096810B5CB0701D5F4
:1001E000002903DA102000F075F910BD4910033121
:1001F00089100022052002F04BF8F6E770B50D6873
:10020000AB0729D1042D27D90F232A684E68134044
:10021000062B0BD12800FFF7B3FF0123984201DA28
:1002200000200AE09A00AE500133F7E7052B13D106
:10023000F30703D4132000F04DF970BD7610FF2EA4
:10024000F8D82800FFF79CFF2C1D80002018A04242
:10025000E6D926700134FAE70B2000F03BF9DFE71E
:1002600070B50C681120E30712D54D68AB072BD190
:10027000042D29D90F262B6864101E40062E0DD19F
:10028000002C04DD2800FFF77BFFA04203DA1220D8
:1002900000F020F901E0A400605970BD331F012B6C
:1002A00012D82800FFF76CFF8000042E02D128002E
:1002B000FFF771FF002CEADDA042E8DB01202C19DA
:1002C000E3785B001843E8E70B20E1E7F8B501238A
:1002D0000D6811201D4214D003244E6834402CD1E7
:1002E000042E2AD90F2332686D108F681340062B15
:1002F0000ED1002D04DD3000FFF742FFA84203DAE3
:10030000122000F0E7F802E0AD00AF512000F8BD88
:10031000052B12D1002DF3DD3000FFF731FF8000F7
:10032000A842EDDB01231F4201D11320E9E77F1032
:10033000FF2FFAD87519EF70E8E70B20E1E708689E
:1003400010B5830717D1042815D90F23026813406D
:10035000062B03D1FFF714FF430004E0052B05D162
:10036000FFF70EFFC3000120184310BD042B02D17C
:10037000FFF711FFF0E70B2000F0ACF8F5E7000005
:1003800002000120104001D0501070470D22014B97
:100390001A70FAE78802002002000120104004D100
:1003A000042A01D91068000970470020FCE770B5E5
:1003B0000E000400FFF7F0FF05003000FFF7ECFF30
:1003C0000023854206D10434AD0004366519AC42E1
:1003D00002D30123180070BD20783278002801D1A3
:1003E000002AF6D0013401369042F0D00023F1E724
:1003F000F0B585B00393019002912D4E2D4B002A4C
:1004000002D002223270013A00251A601B68F554AE
:10041000019B9D4201DB05B0F0BD029AAB00D058B4
:10042000244B1C68C8239B0037191C1B012318424E
:1004300006D0214A43102100380009F005F809E0F0
:100440001E4A002802D004281BD11D4A2100380072
:1004500008F0FAFF300009F05BF8164A039B1060C1
:10046000002B0CD0019B013BAB4208DD154B9842A1
:1004700005D8431C1360202232540022F254013567
:10048000C6E7042810D90F2302681340042B04D1B7
:1004900001F03AFF0C4A0300CDE7062B05D1FFF728
:1004A0007BFF0A4A0300C6E70123094AC3E7C046A7
:1004B00089020020AC0500209DA4000070A400006B
:1004C00076A400001F0300007FB000007BA40000A2
:1004D0008CA40000014B1870002070478802002097
:1004E00070B501F0E9FC094C0100251D1F22280010
:1004F00009F015F8280009F00BF8042304308008EF
:10050000000118432060200070BDC0466402002036
:10051000C368F0B59D00836889B05D190300183386
:1005200006930369069A9F00069B0390DF194369AF
:1005300001939B00D3180293CD4B1B78002B26D13F
:100540007F222B68CB491C1213409B005B5804355B
:1005500001929F46039B587803F094FE0023039A70
:10056000137027E0C24B1B78002B10D12B68019A27
:100570001C121340BF4A9B009B580435E9E7069BB9
:100580003A1DD11ABA4BD82928DD1A221A70039BBA
:10059000B74C9B6821780193EA1A039B92109B78D1
:1005A00012021A43039B587803F074FE0023039A47
:1005B00023701370039B069A9B680193ED1A039BAB
:1005C000AD10DD60069BFE1A039BB6101E61029BF8
:1005D0009B1A039A9B10536109B0F0BD1B783C60D5
:1005E000002B01D01700D2E72B6801991C120B4099
:1005F000A0499B005B5817000435AAE7069B3A1DEB
:10060000D11A9B4BD82902DD1A221A70BFE728683D
:100610001B78291D3860002B02D017000D00B6E7AB
:100620006B6801991C120B4092499B005B581700A4
:1006300008358EE7069B3A1DD11A8D4BD82902DD6D
:100640001A221A70A3E7A4001B782C193C60002B17
:1006500001D017009BE72B6801991C120B408549BC
:100660009B005B581700043573E7069B3A1DD11AAF
:100670007F4BD82902DD1A221A7088E77E49A40030
:1006800061581B783960002B01D017007FE72B6879
:1006900001991C120B4077499B005B5817000435E9
:1006A00057E7043F744B3A68A400E250704B1B7844
:1006B000002B00D06BE72B68019A1C1213406D4A87
:1006C0009B009B58043544E76B4BA400E058FFF7B0
:1006D00057FE043F06003868FFF752FE3618012027
:1006E000654B76000643E650614B1B78002B00D02B
:1006F0004DE72B68019A1C1213405E4A9B009B58E1
:10070000043526E7069B3A1DD11A594BD82902DD3C
:100710001A221A703BE70698029C0121A04202D2DD
:1007200021000C3909681B783960002B01D01700B3
:100730002DE72B6801991C120B404E499B005B581A
:100740001700043505E7069B3A1DD11A484BD829F6
:1007500002DD1A221A701AE70699029881420FD216
:1007600003000C3B1B6845495B106418E41AA400A5
:1007700023583B603E4B1B78002B05D0170006E743
:10078000182119700023F4E72B6801991C120B4003
:1007900038499B005B5817000435DAE6069B029A3D
:1007A000934219D213000C3B1B68344A043FA4182F
:1007B0005B10E31A029A39689B0099502C4B1B7806
:1007C000002B00D0E3E62B68019A1C121340294A43
:1007D0009B009B580435BCE61822254B1A70EDE7A8
:1007E000069B029A93422DD2244B3E1FE31814001D
:1007F0000C3C04932368049A5B10D31A029A9B0062
:100800009858FFF7BDFD07903068FFF7B9FD2468E1
:10081000049B64101C1B079BA4001F1801207F0071
:10082000029B0743E7503700114B1B78002B00D089
:10083000ADE62B68019A1C1213400E4A9B009B5890
:10084000043586E618220A4B1A70EDE7069B3A1D1E
:10085000D11A074BD82902DD1A221A7097E602999D
:10086000A40061581B783960002B09D017008EE670
:100870008802002070A2000070230020FDFFFF3FCF
:100880002B6801991C120B40D8499B005B5817003C
:1008900004355EE6043F029B3A68A400E250D44B64
:1008A0001B78002B00D072E62B68019A1C121340B3
:1008B000CE4A9B009B5804354BE6029BA4001C19B2
:1008C0002368043F38685E10FFF75AFD3618012090
:1008D000C74B76001B7806432660002B00D056E6F7
:1008E0002B68019A1C121340C04A9B009B58043588
:1008F0002FE6069BA4003F1BBD4CBB420CD82378BF
:10090000002B00D043E62B68019A1C121340B74A13
:100910009B009B5804351CE6B64801F069FC23781F
:10092000002B00D033E62B68019A1C121340AF4A0B
:100930009B009B5804350CE6A300ED18002C00DA50
:1009400038E6AB4B1B78002B00D020E62B68019AD1
:100950001C121340A54A9B009B580435F9E5043F3F
:100960003B68042B04D1A300ED18002C00DA21E62B
:100970009F4B1B78002B00D009E62B68019A1C12B4
:1009800013409A4A9B009B580435E2E5043F3B68BC
:10099000042B06D0A200AD18002C02DA002B00D1E7
:1009A00008E6934B1B78002B00D0F0E52B68019AEA
:1009B0001C1213408D4A9B009B580435C9E53A1F11
:1009C00013685B10013B002B06DD01215B00A400D6
:1009D0000B432D191360EDE5854B17001B78002B99
:1009E00000D0D4E52B68019A1C1213407F4A9B006B
:1009F0009B580435ADE53A00069B0C32D31AD82B30
:100A000003DD1A227A4B1A70C1E5FF2361005B00F7
:100A10001940FE3BFF3B19433960039906988968EA
:100A2000241204916D1A0399AD1089782D020D439B
:100A300002999D40091A891099401D430B43BB60E0
:100A4000039B7D609C70E4B26B4BE4000292E35820
:100A5000039A9360664A1278002A03D008331D0077
:100A6000029F94E51D00019A9B680C351C121340EF
:100A70005E4A9B009B58029F6BE53B1F1C68029AD5
:100A8000069B93422FD10A20E3070ED4A30715D16A
:100A9000042C13D90F2322681340042B11D12000FA
:100AA00001F032FC08F034FD0630643003F0D8F871
:100AB00000280FD1043D069B02937BE50720042C00
:100AC000F3D02000431E9841FA234042FF331840E0
:100AD0000730EAE7039B2100587803F0EDFB002381
:100AE000039A1370E7E7029B029A0C3B1B68039979
:100AF0005B109B00D31A0C3B1C601F1D1300083BAE
:100B00001B685A108A70D2B23B49D2005B0055581C
:100B10009B0A039A9B009560ED18029B069A043B82
:100B20001B685B109B00D3180293314B1B78002B82
:100B300000D02CE52B68019A1C1213402B4A9B0015
:100B40009B58043505E53B1F1868FFF719FCA40006
:100B500006003F1B1E2827DC00280DDC244B1B78D9
:100B6000002B00D013E52B68019A1C1213401F4A7A
:100B70009B009B580435ECE401F08CF9033E3618D9
:100B800001F088F91D4B801B9842F9D8184B1B784F
:100B9000002B00D0FBE42B68019A1C121340134A6F
:100BA0009B009B580435D4E40123039A137001F091
:100BB00071F9039B0A3886195E60FBE43B1F1868D5
:100BC000FFF7DEFBA40006003F1B002818DC084BE3
:100BD0001B78002B00D0DAE42B68019A1C1213401A
:100BE000024A9B009B580435B3E4C04670A2000043
:100BF00088020020A0A40000781B00209F8601002E
:100C0000C64B984203DD1D22C54B1A70BFE4012379
:100C1000039A137001F03EF9FA239B005E43039B95
:100C20000A3E30185860C5E4A300FF1A00232000D4
:100C30001A003900FFF7DCFBBA4EBB4C31682000CC
:100C400003F0F2F93168200003F03DFB3168200029
:100C500001F0F0FBB24B1B78002B00D097E42B681F
:100C6000019A1C121340B14A9B009B58043570E452
:100C7000AB4BA4001B783F1B002B00D087E42B68F4
:100C8000019A1C121340A94A9B009B58043560E44A
:100C9000039803F049F8A24B1B78002B00D076E4B0
:100CA0002B68019A1C121340A04A9B009B580435E4
:100CB0004FE43B1F1868002838D1083B1868C30769
:100CC0001ED540103A0001234100083A0B4313603F
:100CD000002859DD01234200391F1A430A603A00F7
:100CE000083A12681A41101A3A000C3A116819426F
:100CF0001FD0C0189840A4001843029BE05027E082
:100D000083070FD104280DD90F2302681340062B47
:100D100002D1FFF741FBD5E7052B03D1FFF73CFBE1
:100D20008000CFE719227E4B1A7030E44010013862
:100D3000CEE78A0723D1042921D90F220E68324039
:100D4000062A15D1013080004358029AA400A3500E
:100D5000734B1B78002B01D0FFF719FC2B68019A0D
:100D60001C121340714A9B009B580435FFF7F1FB9E
:100D7000052A04D108180079A4004000BCE7192214
:100D8000674B1A70FFF703FC0435E1E7A300069AEE
:100D9000FB189B1AD82B13DC0122631E002C14DCD9
:100DA0005F4B1B78002B01D0FFF7F1FB2B68019AFA
:100DB0001C1213405D4A9B009B580435FFF7C9FB8A
:100DC0001A22574B1A70FFF7E2FB3A601C000437F7
:100DD000E3E7069A3B1D9B1A514ED82B03DD1A23DD
:100DE0003370FFF7D4FB069B029AA40093422AD2E9
:100DF0003B1F1868FFF7C4FA011E21DD029B0C3B64
:100E00001A68521082421BDB9007801A484B401828
:100E1000C018029B8000C2583B1B1A60404B3F1B0E
:100E20001B780437002B01D0FFF7B1FB2B68019A28
:100E30001C1213403D4A9B009B580435FFF789FB69
:100E400020233370EAE71823FBE7A3009C46FE1A31
:100E5000002C17DC1C22324B1A70002333606346CF
:100E6000FF1A2F4B04371B78002B01D0FFF78FFBA5
:100E70002B68019A1C1213402C4A9B009B58043586
:100E8000FFF767FB002033685A108300F1580123F5
:100E90000B4003D10D21224A1170DFE749108A422D
:100EA00000DD0A0001308442EFDC012352001343CD
:100EB000D4E7A3009C46FE1A002C17DC1C22184B1A
:100EC0001A70002333606346FF1A154B04371B78F2
:100ED000002B01D0FFF75BFB2B68019A1C1213401B
:100EE000124A9B009B580435FFF733FB0020336800
:100EF0005A108300F15801230B4003D10D21084AF9
:100F00001170DFE749108A4200DA0A00013084429A
:100F1000EFDC012352001343D4E7C04680EE3600D5
:100F200088020020AC0500208902002070A2000089
:100F3000FCFFFF3F3B00083B1868FFF721FA3B1F0F
:100F400006001868FFF71CFA0023864200DA043313
:100F5000A4003A1B17001360E34B04371B78002BE7
:100F600001D0FFF714FB2B68019A1C121340DF4AD3
:100F70009B009B580435FFF7ECFA3B00083B1868D0
:100F8000FFF7FEF93B1F06001868FFF7F9F9F30FAA
:100F9000C217B0425341A4003A1B17009B001360D4
:100FA000D14B04371B78002B01D0FFF7F0FA2B68E8
:100FB000019A1C121340CD4A9B009B580435FFF741
:100FC000C8FA3B00083B18683B1F1968A600BE1B07
:100FD0000423814202D0042802D8002333601CE09D
:100FE0000123184201D01942F7D103239C4618422D
:100FF000F3D102680C331A40042AEED16246114242
:10100000EBD10429E9D90A681340042BE5D1FFF795
:10101000CEF9431E984180003060B34BA4001B788A
:101020003F1B0437002B01D0FFF7B1FA2B68019A60
:101030001C121340AD4A9B009B580435FFF789FAF8
:101040003B00083B18683B1F1968A600BE1B002325
:10105000814202D0042802D8042333601CE001231B
:10106000184201D01942F7D103239C461842F3D10C
:1010700002680C331A40042AEED162461142EBD1C9
:101080000429E9D90A681340042BE5D1FFF78FF949
:101090004342584180003060934BA4001B783F1BB3
:1010A0000437002B01D0FFF772FA2B68019A1C124B
:1010B00013408E4A9B009B580435FFF74AFA3B00C9
:1010C000083B1868FFF75CF93B1F06001868FFF73C
:1010D00057F9F317C20F86425341A4003A1B170079
:1010E0009B001360804B04371B78002B01D0FFF767
:1010F0004EFA2B68019A1C1213407C4A9B009B58A5
:101100000435FFF726FA3B00083B1868FFF738F96B
:101110003B1F06001868FFF733F90023864200DD05
:101120000433A4003A1B170013606F4B04371B787D
:10113000002B01D0FFF72BFA2B68019A1C121340E9
:101140006A4A9B009B580435FFF703FA3B1F1B6854
:10115000A400043B5A1E93413A1B17009B001360E6
:10116000614B04371B78002B01D0FFF710FA2B6876
:10117000019A1C1213405D4A9B009B580435FFF7EF
:10118000E8F93B00083B1868FFF7FAF83B1F060038
:101190001868FFF7F5F832180120A4003B1B1F0068
:1011A000520002431A60504B04371B78002B01D0C9
:1011B000FFF7EDF92B68019A1C1213404B4A9B0074
:1011C0009B580435FFF7C5F93B00083B1868FFF74B
:1011D000D7F83B1F06001868FFF7D2F8321A012033
:1011E000A4003B1B1F00520002431A603E4B043711
:1011F0001B78002B01D0FFF7CAF92B68019A1C124B
:1012000013403A4A9B009B580435FFF7A2F93B0074
:10121000083B1868FFF7B4F83B1F06001868FFF793
:10122000AFF802000120A4003B1B1F0072435200D4
:1012300002431A602C4B04371B78002B01D0FFF7B8
:10124000A6F92B68019A1C121340284A9B009B5850
:101250000435FFF77EF93B1F1868FFF791F8061E6B
:1012600017D11F22204B1A70A4003B1B1F001E60C9
:101270001D4B04371B78002B01D0FFF788F92B6832
:10128000019A1C121340194A9B009B580435FFF722
:1012900060F93B00083B1868FFF772F8310005F071
:1012A000E5FE012640000643DEE73B1F1868FFF716
:1012B00067F8061E1CD11F220B4B1A70A4003B1BA3
:1012C0001F001E60084B04371B78002B01D0FFF76E
:1012D0005EF92B68019A1C121340044A9B009B582C
:1012E0000435FFF736F9C0468802002070A20000DE
:1012F0003B00083B1868FFF743F8310005F09CFFFE
:10130000012649000E43D9E73B1F1868FFF738F85C
:10131000C217801850400122A4003B1B1F00400050
:1013200010431860F14B04371B78002B01D0FFF7F6
:101330002EF92B68019A1C121340ED4A9B009B5812
:101340000435FFF706F9A300FE1A3068012C24D1FA
:10135000FFF716F80494079008F032F8079900296F
:1013600000DC012105F068FF049BA400C9180123DB
:1013700049001943DD4B3F1B1B7831600437002BBC
:1013800001D0FFF704F92B68019A1C121340D84AC8
:101390009B009B580435FFF7DCF8FEF7F1FF049043
:1013A0007068FEF7EDFF049B0130C31A0793D3E783
:1013B000A300FE1A31002000049300F0DBFF049B21
:1013C0003060FF1AC94B04371B78002B01D0FFF7A0
:1013D000DEF82B68019A1C121340C54A9B009B58EB
:1013E0000435FFF7B6F83B00083B1868FEF7C8FF66
:1013F0003B1F06001868FEF7C3FF02000120A4008F
:101400003B1B1F003240520002431A60B74B0437A7
:101410001B78002B01D0FFF7BAF82B68019A1C1239
:101420001340B34A9B009B580435FFF792F83B00EA
:10143000083B1868FEF7A4FF06003B1F1868FEF77C
:101440009FFF320002430120A4003B1B1F005200FB
:1014500002431A60A54B04371B78002B01D0FFF71D
:1014600096F82B68019A1C121340A14A9B009B58C6
:101470000435FFF76EF83B00083B1868FEF780FF65
:1014800006003B1F1868FEF77BFF32004240012038
:10149000A4003B1B1F00520002431A60934B043709
:1014A0001B78002B01D0FFF772F82B68019A1C12F1
:1014B00013408F4A9B009B580435FFF74AF83B1FA7
:1014C0001868FEF75DFFC0430122A4003B1B1F000C
:1014D000400010431860854B04371B78002B01D067
:1014E000FFF755F82B68019A1C121340804A9B00A5
:1014F0009B580435FFF72DF83B00083B1868FEF7B2
:101500003FFF06003B1F1868FEF73AFF320082409B
:1015100051000122A4003B1B1F000A431A60734BB9
:1015200004371B78002B01D0FFF731F82B68019AA4
:101530001C1213406E4A9B009B580435FFF709F8B4
:101540003B00083B1868FEF71BFF06003B1F1868AE
:10155000FEF716FF3200024151000122A4003B1B9E
:101560001F000A431A60614B04371B78002B01D01F
:10157000FFF70DF82B68019A1C1213405C4A9B0080
:101580009B580435FEF7E5FF3B000C3B1868FEF75F
:10159000F7FE3B00083B06001868FEF7F1FEF11766
:1015A0000200C317300005F099FE3B1F049005911F
:1015B0001868FEF7E5FE02000498059905F042FE62
:1015C00043000120A4003E1B37001843474B306006
:1015D0001B780437002B01D0FEF7D9FF2B68019A46
:1015E0001C121340424A9B009B580435FEF7B1FF82
:1015F000A300FE1A310020000493FEF7DDFD049BDA
:101600003060FF1A394B04371B78002B01D0FEF7EE
:10161000BEFF2B68019A1C121340354A9B009B5851
:101620000435FEF796FFA300FE1A31002000049354
:10163000FEF7D2FD049B3060FF1A2C4B04371B7859
:10164000002B01D0FEF7A3FF2B68019A1C12134058
:10165000274A9B009B580435FEF77BFFA300FF1A27
:1016600039002000FEF7CAFD204B1B78002B01D06B
:10167000FEF78DFF2B68019A1C1213401C4A9B0039
:101680009B580435FEF765FFA300FE1A31002000C9
:101690000493FEF7E5FD049B3060FF1A134B0437FB
:1016A0001B78002B01D0FEF772FF2B68019A1C12E9
:1016B00013400F4A9B009B580435FEF74AFFA300D6
:1016C000FF1A39002000FEF701FE084B1B78002BA3
:1016D00001D0FEF75CFF2B68019A1C121340044AEC
:1016E0009B009B580435FEF734FFC046880200205B
:1016F00070A20000A300FE1A310020000493FEF740
:101700001EFE049B3060FF1AF24B04371B78002B3F
:1017100001D0FEF73CFF2B68019A1C121340EE4AE1
:101720009B009B580435FEF714FF069B3E1DF31AE1
:10173000E84CD82B03DD1A232370FEF728FF00F0B6
:10174000B3FB43000120184323783860002B02D0FC
:101750003700FEF71CFF2B68019A1C121340DE4A6B
:101760009B009B5837000435FEF7F3FE069B3E1D99
:10177000F31AD84CD82B03DD1A232370FEF707FF8A
:1017800000F088FBD54B4000184001231843237814
:101790003860002B02D03700FEF7F9FE2B68019A63
:1017A0001C121340CC4A9B009B5837000435FEF7AF
:1017B000D0FE0123A600BE1B20001A003100FEF758
:1017C00017FEC74C2068643002F04AFA002802D1A4
:1017D000043DFEF7EFFE039B21685A78C14802F0F2
:1017E00080FD0123039A3700137000F053FBBE4BBA
:1017F00022681B68063253431818039B5860FEF793
:10180000D9FEA600BE1B2000012300223100FEF7F6
:10181000EFFDB34C2068643002F022FA0028D7D0E4
:10182000B04802F059FBDCE7A4003E1BFEF758FE6F
:101830003700A84B30601B780437002B01D0FEF72F
:10184000A6FE2B68019A1C121340A34A9B009B58CA
:101850000435FEF77EFEA4003E1B300000F053FB73
:1018600037009C4B30601B780437002B01D0FEF70B
:101870008EFE2B68019A1C121340974A9B009B58BE
:101880000435FEF766FEA4003E1B300000F03DFB71
:101890003700904B30601B780437002B01D0FEF7E7
:1018A00076FE2B68019A1C1213408B4A9B009B58B2
:1018B0000435FEF74EFEA300FE1A3100200004930B
:1018C00000F026FB049B3060FF1A824B04371B7824
:1018D000002B01D0FEF75BFE2B68019A1C1213400F
:1018E0007D4A9B009B580435FEF733FEA4003F1B46
:1018F000380000F03FFB774B1B78002B01D0FEF740
:1019000046FE2B68019A1C121340734A9B009B5899
:101910000435FEF71EFEA300FE1A310020000493DA
:1019200000F050FB049B3060FF1A6A4B04371B78B1
:10193000002B01D0FEF72BFE2B68019A1C121340DE
:10194000654A9B009B580435FEF703FEA4003F1B2D
:10195000380000F079FB5F4B1B78002B01D0FEF7BD
:1019600016FE2B68019A1C1213405B4A9B009B5881
:101970000435FEF7EEFD0121200000F04DFB554B34
:101980001B78002B01D0FEF702FE2B68019A1C1277
:101990001340514A9B009B580435FEF7DAFD0021A5
:1019A000200000F039FB4B4B1B78002B01D0FEF7D9
:1019B000EEFD2B68019A1C121340474A9B009B586E
:1019C0000435FEF7C6FDA4003E1B300000F05EFBB0
:1019D0003700404B30601B780437002B01D0FEF7F6
:1019E000D6FD2B68019A1C1213403B4A9B009B5862
:1019F0000435FEF7AEFDA4003E1B300000F05AFB9C
:101A00003700344B30601B780437002B01D0FEF7D1
:101A1000BEFD2B68019A1C1213402F4A9B009B5855
:101A20000435FEF796FDA4003F1B380000F01CFBB8
:101A3000284B1B78002B01D0FEF7A9FD2B68019ADB
:101A40001C121340244A9B009B580435FEF781FD6D
:101A5000A4003F1B380002F02BFF1E4B1B78002B0D
:101A600001D0FEF794FD2B68019A1C1213401A4A0C
:101A70009B009B580435FEF76CFDA4003E1B300014
:101A800002F0A8FF3700134B30601B780437002B9F
:101A900001D0FEF77CFD2B68019A1C1213400E4A00
:101AA0009B009B580435FEF754FDA4003F1B3800F3
:101AB00002F0AEFE074B1B78002B01D0FEF767FD4E
:101AC0002B68019A1C121340034A9B009B58043553
:101AD000FEF73FFD8802002070A20000FEFFFF7F9E
:101AE000AC0500208902002004000020A4003E1B59
:101AF000300002F0A3FE3700B14B30601B78043792
:101B0000002B01D0FEF743FD2B68019A1C121340F5
:101B1000AC4A9B009B580435FEF71BFDA300FF1A3F
:101B20003900200000F0FCFEA54B1B78002B01D0F3
:101B3000FEF72DFD2B68019A1C121340A14A9B0051
:101B40009B580435FEF705FDA300FF1A390020005D
:101B500000F06EFD9A4B1B78002B01D0FEF717FDAD
:101B60002B68019A1C121340964A9B009B5804351F
:101B7000FEF7EFFCA300FF1A3900200000F068FD1B
:101B80008F4B1B78002B01D0FEF701FD2B68019ACB
:101B90001C1213408B4A9B009B580435FEF7D9FC5E
:101BA000A300FF1A3900200000F07AFD844B1B7857
:101BB000002B01D0FEF7EBFC2B68019A1C1213409E
:101BC000804A9B009B580435FEF7C3FCA300FE1A15
:101BD00031002000049302F087FF049B3060FF1A5D
:101BE000774B04371B78002B01D0FEF7D0FC2B6815
:101BF000019A1C121340734A9B009B580435FEF750
:101C0000A8FCA300FE1A31002000049302F074FF28
:101C1000049B3060FF1A6A4B04371B78002B01D0FD
:101C2000FEF7B5FC2B68019A1C121340654A9B0015
:101C30009B580435FEF78DFCA300FE1A31002000EE
:101C4000049302F061FF049B3060FF1A5C4B043781
:101C50001B78002B01D0FEF79AFC2B68019A1C120E
:101C60001340584A9B009B580435FEF772FCA300B2
:101C7000FE1A31002000049302F082FD049B3060C4
:101C8000FF1A4F4B04371B78002B01D0FEF77FFC67
:101C90002B68019A1C1213404A4A9B009B5804353A
:101CA000FEF757FCA300FF1A3900200000F0DAFD10
:101CB000434B1B78002B01D0FEF769FC2B68019A7F
:101CC0001C1213403F4A9B009B580435FEF741FC11
:101CD000A300FF1A3900200000F00AFD384B1B78E2
:101CE000002B01D0FEF753FC2B68019A1C12134005
:101CF000344A9B009B580435FEF72BFCA300FE1AC8
:101D000031002000049300F021FE049B3060FF1A94
:101D10002B4B04371B78002B01D0FEF738FC2B68C7
:101D2000019A1C121340274A9B009B580435FEF76A
:101D300010FCA300FF1A3900200000F079FD204BB1
:101D40001B78002B01D0FEF722FC2B68019A1C1295
:101D500013401C4A9B009B580435FEF7FAFBA30076
:101D6000FF1A3900200001F001FF154B1B78002BF2
:101D700001D0FEF70CFC2B68019A1C121340114A8B
:101D80009B009B580435FEF7E4FBA300FE1A3100CC
:101D90002000049301F0EAFE049B3060FF1A084B18
:101DA00004371B78002B01D0FEF7F1FB2B68019A5A
:101DB0001C121340034A9B009B580435FEF7C9FBD5
:101DC0008802002070A200000023F7B55A1E01927D
:101DD000002B07DA00F0EEFD02F080F902F0D8FAED
:101DE0006423019300263000194B1968B14212DDBB
:101DF000184B1A6801328A420FDAF0241A601D6803
:101E0000154F6C43E35D002B1FD0E419022B06D164
:101E10002000FEF77DFB019BD8E70022EDE7012BB8
:101E20000DD1002801D100F035F8F0226A43BB182B
:101E30005B680A49C31A8B4201D80223BB54F023C2
:101E40005D43054BEB5C022BE2D00136CCE7C0468C
:101E5000B005002000000020181200209F8601001D
:101E60000020704700207047002070470020704716
:101E700001220020054B06491A61585004310330F5
:101E800058500831801858501A6070470080004040
:101E9000040500000122034B1A64A822D2009858BE
:101EA0007047C0460080004010B5FFF7F3FFFA21ED
:101EB000890005F051F810BD00487047F0A40000FB
:101EC0001D20704770B5054E0400335C0D008B4239
:101ED00002D003F02BFD355570BDC046B40500207F
:101EE00070B50024064D635D012B05D10021200053
:101EF00003F01CFD0023635501341D2CF2D170BD8D
:101F0000B405002070470D2070473B20704700004B
:101F1000F8B501240B6806000D00234204D10D2002
:101F2000FEF7D8FA2000F8BD5B102000052BFAD888
:101F30000E4A9B009C580E4F3B5D002B05D00021A4
:101F4000200003F0F3FC00233B55012E06DD6B68F7
:101F5000042B03D10221200003F0E8FC200003F051
:101F600093FB012440002043DDE7C046D8A40000D5
:101F7000B4050020F8B501260568354202D0446852
:101F8000344203D10D20FEF7A5FAF8BD6D101C2DCB
:101F9000FBD80A4F7B5D012B04D03100280003F0F1
:101FA000C5FC7E55064964108C4202DCE143C9172A
:101FB0002140280003F0EEFBE7E7C046B40500200F
:101FC000FF03000070B501240D68254204D10D20E7
:101FD000FEF780FA200070BD6D101C2D17D800246C
:101FE000012804DD4C68043C63425C416400094EF6
:101FF000735DA34204D02100280003F097FC7455C0
:10200000280003F0C7FC03000420012BE3D00020CC
:10201000E1E7C046B405002070B504000D001C289F
:102020000ED8084E335C012B04D0012103F07EFC56
:1020300001233355290020004D1EA94103F094FCD3
:1020400070BDC046B4050020036810B5DA0703D49C
:102050000D20FEF73FFA10BD4168581004394A427E
:102060005141FFF7D9FFF6E737B569460A00064B3D
:1020700030CB30C203680220042B02D100F0E8FA12
:1020800037BD00F00DFBFBE7B0A4000010B5084C15
:102090006379002B05D00021052003F047FC0023C5
:1020A0006371052003F076FC43425841800010BD67
:1020B000B405002010B5084CE37A002B05D00021B0
:1020C0000B2003F033FC0023E3720B2003F062FCCF
:1020D00043425841800010BDB4050020704770474E
:1020E00010B5034A0421034801F02CFD10BDC04681
:1020F000B8A40000B8AB0000E12170B54902144853
:1021000003F0BAF8FFF7B4FE0A2003F0B7FA002391
:10211000FF21104A995401331D2BFBD101220020CD
:102120000D4B01001A6004230C4A0D4D1468002C5D
:10213000FCD02C680002013B20431160002BF5D13C
:102140000122084B1A6003F053FA00F07FFD70BDC6
:10215000A0110020B405002000D0004000D10040B4
:1021600008D5004004D00040F8B50B4E0700300001
:102170000D0003F0C9F80400A84200DD2C003D006A
:10218000EB1B9C4205DD300003F0C8F828700135D8
:10219000F6E72000F8BDC046A011002010B50100F0
:1021A000014803F071F810BDA011002010B5054CD6
:1021B000200003F077F8E1212000490203F05CF8E9
:1021C00010BDC046A0110020064B01201A68064B26
:1021D00006491A6000239A0001338850642BFAD113
:1021E0007047C046DC050020D40500207023002085
:1021F00000B59BB00200054901A807F057F901A8F6
:1022000001F086FE02F0C4F8FCE7C04677A50000A6
:1022100037B5184D04002868002801D006F034FDB9
:10222000A400200006F026FD2860002802D11248F4
:10223000FFF7DEFF01AB984207D2104B02196B4447
:102240000193934201D20E48F2E7042802D80830E5
:102250002860083C2B680B4A1C1913600A4B0120AC
:102260001C60002309499A0001338850642BFAD17D
:1022700037BDC046DC0500201DA500001CFCFFFF8B
:102280004DA50000D4050020D805002070230020B3
:1022900070B50D4D0D4E04004B1C28689B00366830
:1022A000C318B34203D90A20FEF714F970BD2B609E
:1022B0000500AB4205D80F2309011C4021430160F2
:1022C000F4E704C5F5E7C046D4050020D805002092
:1022D0000322CB1C70B50C00D9171140C91805009A
:1022E000891000220420FFF7D3FF0023A34206DB5E
:1022F000E343DB171C4000230419237170BDE95C24
:10230000C21811710133F1E710B5830706D1042813
:1023100004D90F2208C81340042B03D00E20FEF767
:10232000D9F8014810BDC04687A5000010B50124AA
:102330000B681C4016D05C10200005F02BF90B49EF
:1023400004F0F6FF06F0BEFB03F068FC0022084B29
:1023500005F08EFD03F00AFC06F044FB430001206B
:10236000184310BD0D20FEF7B5F8E5E7D302373965
:102370000000D04010B503240868044006D10428AA
:1023800004D90F2302681340042B03D00E20FEF75C
:10239000A1F810BDFFF7B8FF03782100233B5A4294
:1023A00053411022C01807F051F980239B05C21831
:1023B000044B9A4201D91420E9E743000120184355
:1023C000E7E7C046FFFFFF3F10B5034A022103487D
:1023D00001F0B8FB10BDC04690A5000088A5000024
:1023E0000020704710B51E20FEF774F810BD10B520
:1023F0001E20FEF76FF810BD10B51E20FEF76AF81C
:1024000010BD10B51E20FEF765F810BD10B51E20DA
:10241000FEF760F810BD10B51E20FEF75BF810BD8A
:1024200010B51E20FEF756F810BD10B51E20FEF7A1
:1024300051F810BD7047000010B5034A0921034848
:1024400001F080FB10BDC046B0A50000F8A500005B
:102450000120034B1860034B1B68834018437047EF
:1024600000060020E0050020F0B5EFF31081012305
:10247000194083F31088134C134AA4461268134E74
:10248000013A9340124F134A002B17D014680342AD
:102490000FD03D682C60C046C046C046C046C0460E
:1024A000C046C046C0460C4C1568246825605B08D1
:1024B000EAE765462C6014683460F8E781F3108819
:1024C000F0BDC04608050050080000200C05005073
:1024D000EC050020F4050020E805002030B585B0AB
:1024E00001AD0C220649280006F0D8FB0024285D27
:1024F00001210134FFF7E6FC0C2CF8D105B030BD0A
:1025000084A60000F0B585B06A463C4B3C49138078
:102510001C2301AF93700C310922380006F0BEFB7A
:10252000FFF7C2FC374B384DC0182B68984201D2D8
:1025300000232B602C68002C44D13E5D012130002B
:10254000FFF7C0FC01340121300003F00DFA092C23
:10255000F3D100246B461E5D01213000FFF7B2FC71
:1025600001340021300003F0FFF9032CF2D1C82020
:1025700080000138C046C046C046C046C046C0467E
:10258000C046C046C046C046C046C046F1D1002144
:102590000420FFF797FC6B4600211878FFF792FCA8
:1025A0006B4600215878FFF78DFC6B460021987828
:1025B000FFF788FCFFF778FC002413302860200028
:1025C00005B0F0BDFFF770FC2B6800249842F6D3ED
:1025D000042003F059F80D4B0D4EC0180BD4306099
:1025E0003068032104F042FD00230A4A30602B606A
:1025F00013600124E3E73460F2E7C0461A1B0000D1
:1026000084A6000010270000F8050020C8FEFFFF88
:10261000E00500200006002010B50124044002D08F
:102620004410200010BD0D20FDF754FFF9E7000015
:102630000022054B10B51A60044B1B68934201D071
:1026400002F0C8FA002010BDFC050020C4100020D4
:1026500070B508680D00FFF7DFFF04006868FFF73A
:10266000DBFF621E0100042A14D8451E042D11D878
:1026700005236B439B18012215009D402B00064843
:1026800005682B430360054B1B68002B02D020001C
:1026900002F0A1FA002070BDFC050020C41000204B
:1026A00070B508680D00FFF7B7FF04006868FFF712
:1026B000B3FF621E0100042A13D8451E042D10D852
:1026C00005236B439B1801229A40074803689343F4
:1026D0000360064B1B68002B03D00022200002F091
:1026E0007AFA002070BDC046FC050020C41000200E
:1026F000F0B5050089B008680C00FFF78DFF069063
:10270000022D36DD6068FFF787FF0190A068FFF7B4
:1027100083FF04000127231D661E0793731C029389
:10272000079B9E4235D0052373430593019B019D72
:1027300005330493049BAB421ED0042E16D86B1EA7
:10274000042B13D80122059B2349013B5B199A40B6
:102750009446224A0B681068069A3A4003920DD0BC
:1027600062461A430A60012200280DD17F0001351C
:10277000E0E701240194CDE7029ECFE76246934350
:102780000B600028F2D0039A0299280002F023FA85
:10279000ECE7019B1E1D042E1AD8012C18D1002530
:1027A00005273B0021006B439B1999400B000A4A07
:1027B000013511689943094B11601B68002B05D046
:1027C000019B0022581D290002F005FA052DE8D1D1
:1027D000002009B0F0BDC046FC050020C410002058
:1027E00010B5041E10DA00240A4BA400E25801239D
:1027F0009340094A09491360094A1160094A0A4984
:1028000011600A4A136010BDFFF75AFBA042EADDCF
:10281000EAE7C046F8B20000F405002008050050C1
:10282000EC050020E80500200C05005018050050BC
:102830000200086810B5C3070FD540101823012AFD
:1028400003DD4A68042A00D10833054A1360FFF704
:1028500059FBFFF7C5FF002010BD01204042EDE706
:10286000080000202B4BF7B51B680C00002B03D190
:1028700001204042FFF7B4FF0126246834421AD0F9
:10288000FF226310120260121040DAB21043FF22DE
:102890001B021204134018431F4B1B68202B06D148
:1028A000B4401E4BA40EA400E35800021843FFF7E7
:1028B000DBFD0020FEBD03252540FAD1042CF8D90C
:1028C0000F2322681340062BF3D1FF27130901932E
:1028D0003F02019B9D42ECDA0135AB00E3583342E5
:1028E000F7D05A105812D1B238400843FF211202D3
:1028F00009040A401043084A1268202A06D15B00E6
:102900009B0E06499B00020258581043FFF7ACFD8E
:10291000DFE7C046F40500200800002074A800008E
:10292000086810B5C30703D5FFF776FE054B18609E
:10293000054B1B68002B03D0024B186802F04CF9C2
:10294000002010BDFC050020C41000200868F8B568
:10295000C3071AD5FFF760FE0300203B5E2B25D886
:102960000520012258430023114E451DA84219D0CD
:1029700005211024375C3C4200D09B1801395200DD
:1029800064100029F7D10130F0E783070ED1042845
:102990000CD90F2203681A40042A07D11B0905D05D
:1029A0000079D9E701205B001843F8BD0120FCE75E
:1029B00099A600007FB5A04C2368002B0AD19F4A3E
:1029C0001268002A06D19E4B1B68002B01D0FFF72E
:1029D00099FD7FBD9B4D2A68002A26D1984A12682E
:1029E000002A1BD0FFF78EFD0028F2D0FFF776FDFE
:1029F000924B24681A681C60002A16D0002C14D14F
:102A000001AD0C229049280006F048F9285D00210C
:102A10000134FFF757FA0C2CF8D1DAE7874A12682D
:102A2000002AE5D1002BE3D0E0E700211A2002F0D4
:102A30009BFF00211B2002F097FF00211C2002F0C9
:102A400093FF2E68012E5CD0022E00D1A2E0002E52
:102A500050D101363100794C03202368994302F0AC
:102A600083FF0420216801404B42594102F07CFF62
:102A7000102123680A2019404B42594102F074FF8B
:102A800080212368090119404B425941062002F078
:102A90006BFF80212368090219404B4259410720EE
:102AA00002F062FF80212368490219404B425941DC
:102AB000092002F059FF80212368890219404B4206
:102AC0005941192002F050FF80212368C9021940A2
:102AD0004B425941182002F047FF802321681B0315
:102AE00019404B425941172002F03EFF31001A2095
:102AF00002F03AFF2B680321581C04F09DFB29606B
:102B000067E702214D4C1720236819404B42594179
:102B100002F02AFF08212368182019404B4259412E
:102B200002F022FF80212368C90019404B4259411D
:102B3000042002F019FF80212368490119404B420B
:102B400059410A2002F010FF80212368C901194071
:102B50004B425941032002F007FF8021236889037B
:102B600019404B425941092002F0FEFE80232168A2
:102B70001B0419404B425941192002F0F5FE310067
:102B8000062002F0F1FE3100072002F0EDFE3100D8
:102B90001B20ADE72021294C1720236819404B4208
:102BA000594102F0E1FE40212368182019404B42B0
:102BB000594102F0D9FE80212368192019404B4267
:102BC000594102F0D1FE80212368490019404B424F
:102BD0005941092002F0C8FE80212368890019406C
:102BE0004B425941072002F0BFFE80212368890132
:102BF00019404B425941062002F0B6FE802123685D
:102C0000490319404B4259410A2002F0ADFE802190
:102C10002368C90319404B425941032002F0A4FE26
:102C2000802321685B0419404B425941042002F083
:102C30009BFE01211C205BE7FC050020F005002025
:102C400000060020E405002084A60000012010B545
:102C50004042FFF7C5FD10BD10B5034A09210348E6
:102C600000F070FF10BDC04674A90000BCA90000B0
:102C700030B502248025094B094AED009C505C596F
:102C8000002CFCD0A124E400884202D300219950FA
:102C900030BD8025ED0018514019F5E700E00140F6
:102CA0000405000010B5002806D1C020B021400264
:102CB0008902FFF7DDFF10BDB02080218002C9022C
:102CC000F7E7000043425841064B40421840B0230A
:102CD0009B02C018036800201A0E532A01D11B0260
:102CE000180A704700C0FEFF30B501248025054B4F
:102CF000054AED009C505C59002CFCD0016000217D
:102D0000995030BD00E001400405000043425841A5
:102D1000074B40421840B0239B02C018A62310B5B1
:102D20000902DB05090A1943FFF7DEFF10BDC046A3
:102D300000C0FEFF70B5012480250D4B0D4EED0047
:102D40009C515C59002CFCD0002902DC00229A51D5
:102D500070BD557814782D022543947801392404E8
:102D60002543D478043224062C4310C0ECE7C04637
:102D700000E001400405000070B505004B680A0042
:102D80009C1C2100A400FFF7D5FF281970BD00008E
:102D9000134B1B68002B0CD08022B023D2029B0265
:102DA00000280BD11A1D5B681B0E522B00D110009E
:102DB0007047B022C02392025B02F1E782420DD934
:102DC00003681B0E522B09D1436802339B00C018C5
:102DD000824203D903681B0E522BE9D00020E7E79B
:102DE0000407002070B50020FFF7D2FFFF26050082
:102DF000002801D1280070BD03681C143440FFF77F
:102E0000C7FFDA2CF4D10500F2E700008022F0B50C
:102E10005200A1B00021674805F049FF802200213F
:102E20005200654805F043FF644BFF271B681A00FA
:102E3000049353425A4110000592FFF733FF049C5C
:102E40000020631E9C415E4B64421C405D4BE418B5
:102E5000FFF7C8FF0600002E2DD10498FFF732FFC0
:102E6000411C0598FFF752FF059A574D534B2C60B4
:102E70001A60FFF79BF9514B64201B68A0215A424E
:102E800053414F4A5B421340B0222C6892029B1878
:102E9000E41A6043490204F0E9F8A0225202030058
:102EA00000924A49220007A806F000FB07A801F09B
:102EB0002FF821B0F0BD3268131412123A403B4093
:102EC00003921A000A3A092A49D83A4B039A995CA4
:102ED000002931D110223E4805F0E9FE35002B686B
:102EE00003991A123A40914209D11A143A400B2A16
:102EF00027D0132A2DD00A2A01D1354B1D60280076
:102F0000FFF746FF051EEAD1314B196800290FD0A3
:102F10002000FFF731FF04002D4B5B195968002991
:102F200003D02000FFF728FF040004350C2DF3D157
:102F3000204B0121039A99543000FFF729FF060026
:102F400089E73B40022BDADC214A9B00D3185D6005
:102F5000D5E7102200211E4805F0A9FECFE71A0090
:102F6000153A082AE8D8144A0399525C002AE3D19A
:102F70003500152B00D01500300003681A143A40B4
:102F8000152A0FD01D2A00D10025FFF701FF0028C8
:102F9000F3D1002D04D020002900FFF7EDFE04003E
:102FA000054BC6E7039A1B123B409A42EDD1050040
:102FB000EBE7C046040600200C07002004070020B1
:102FC00000C0FEFF04C002000807002055AA000050
:102FD00000250020F0B50020B7B00024FFF7D8FE90
:102FE000270005002600002D2ED1284D2868FFF768
:102FF00069FE32003B0001900094254904A806F0C8
:1030000055FA04A800F084FF224B64201C682B684A
:10301000A0215A425341204A5B421340B0229202FF
:103020009B18E41A6043490204F020F8A0225202DF
:10303000030000921949220004A806F037FA04A8F8
:1030400000F066FF37B0F0BDFF226B6829689C4630
:103050000233FF180B12013613409C4200DA1C00A9
:10306000FF200A140240039262460140019200913F
:10307000039A0B4904A806F019FA04A800F048FFC7
:103080002800FFF785FE0500ADE7C04604070020D5
:10309000C6AA00000807002000C0FEFF70AA0000BA
:1030A000B2AA000070B50020FFF70CFE040001205A
:1030B000FFF708FE844200DA04000A4B1D686A42EA
:1030C000554128001D60FFF7EDFDA0226B42520222
:1030D0001340054A28009B18044A611C1360FFF73F
:1030E00015FE70BD040700200480010008070020C1
:1030F000F8B50020FFF7E6FD07000120FFF7E2FD2D
:103100003E00204D0643204C0DD18021C020C90235
:103110004002FFF7ADFD01213000FFF7F7FD1B4B2B
:103120002E6023601DE0874209DD0023B0212B6063
:10313000164B8902236023680020012517E0012334
:1031400080212B60124BC9022360F4E7120E522A31
:1031500008D0002800D023600E4800F0D9FEFFF709
:10316000A1FFF8BD28005A68023292009B188B42DA
:1031700005D21A68561CE9D10028F2D0D1E72160A7
:10318000EFE7C04604070020080700200480010084
:1031900004C002008BAA0000F0B585B003920322A0
:1031A0000333DC17294D1440E4182B68284F5A428A
:1031B000534180225B42D202A4103B409B18A21CC8
:1031C0000291244E910000910190316800980A18F4
:1031D000934215D2FFF71AFE2B685A4253418022C0
:1031E0005B421F40D202BF183368009A9B189F426F
:1031F00006D2194800F08CFE0025280005B0F0BD6D
:10320000029B356819066B461A7BA423DB05134322
:10321000FF222F00090C1943019B12041B041340C9
:1032200019432800FFF760FD0837281D210037608B
:10323000FFF75AFD002C04D00A9A21003800FFF74E
:1032400079FD009B083BFF183760D6E70407002094
:1032500000C0FEFF080700202FAA000010B5FFF7EE
:10326000D5FD10BD70B59AB0FFF742FFFF221E4C8E
:10327000D2000021200005F01AFDFF25FFF7B2FD66
:103280000026002814D10200C300E3580130591E63
:103290008B41D218FF28F7D1144901A806F006F98E
:1032A00001A800F035FE124800F032FE1AB070BDE1
:1032B00003681A142A400A2A0AD11A122A40FF2A3D
:1032C00003D0D200A1180B71A050FFF761FDD8E721
:1032D000132AFAD11B122B40FF2BF6D0DB00E21889
:1032E0001671E650F1E7C046781B0020FBAA0000EB
:1032F0000FAB00000021094B094A596001315160B0
:1033000059680029FCD00021196101239360022231
:10331000044B8131FF315A501A607047FC10004055
:103320000010004000E100E00222064B0121DA67B4
:103330000022054B5A61054A11615A69002AFCD0E6
:103340007047C04604E100E0FC100040001000405F
:1033500010B5044C2378002B01D0FFF7E5FF0020C7
:10336000207010BD0D0800200120024B1B685B007F
:10337000184370479008002003480368002B02D1CF
:103380001422037102607047282500200120024B9F
:103390001B685B00184370470C00002070B50400E8
:1033A0000D001600FEF780FD8023012200215B0541
:1033B0005B6E6270E270020AA271020CE2711A0A7C
:1033C00060716372000EA2721A0C1B0E26702571BA
:1033D000A1702072E272237370BD0000124B10B511
:1033E0001B68124C5A1C0FD0114C002B0CD0114CE6
:1033F000012B09D0104C022B06D00D4C042B03D00E
:103400000E4C052B00D10B4C21000D4806F078F82E
:10341000200006F07DF80300042204339B080948CD
:103420001B011343036010BD1000002097AB000088
:1034300090AB0000A2AB0000A7AB00009CAB00006B
:10344000142500201025002070B5214C2278002A78
:103450003DD1204B01215A608022D20511605A686B
:10346000002AFCD0002207201B4B1C4901255A5082
:103470000439585008315A5019481A4958501A49B5
:103480001A485A501A495A50A622D2009D50082272
:1034900018495A50043158500220174958501749BA
:1034A0001748585017480439585018201649585092
:1034B000C12189005A500539FF39585892180243E2
:1034C0005A501249124A9950FFF714FF257070BDE7
:1034D0000D080020FC000040001000400C0500001A
:1034E000746962751C0500002405000020000402B8
:1034F0002C05000014050000340500003C05000008
:10350000FFFF000021100100540500000E080020FC
:103510000405000070B50E4B06001B78002B01D18E
:10352000FFF792FF00200B4D2C7884420ED00A4BFF
:10353000202219780323091B1940084B4901C91897
:10354000300005F0ABFB0120013C2C7070BDC04683
:103550000D080020940800200C0800200E08002010
:10356000002330B589B0984225DD03240D682C4036
:103570009C4220D12300042D1DD90F212A6811401F
:10358000062918D112091F2A15D96846FFF7C2FF6C
:10359000230000280FD06B46012218781300A042A8
:1035A00003DB6B461B5D5B0013430134A1006B50D2
:1035B000202CF3D10423180009B030BD70B5414B65
:1035C0008AB01B78002B01D1FFF73EFF02AD280027
:1035D000FFF7A0FF002802D100200AB070BD2B78B1
:1035E0000B2BF9D96B78012BF6D1EB78012BF3D1AA
:1035F0000023354E354C336023712B79344A1360E8
:10360000002B0ED1152169444A780B7812021A4317
:103610008B781B041A43CB781B06134333600023BB
:1036200018E0012B20D1152169444A780B78120249
:103630001A438B781B041A43CB781A211B061343B9
:1036400033600E236A7C6944934200DD130000223C
:103650009A4232D104200021E21804339B101B014E
:10366000034311712360B8E7022B03D16A7B103347
:103670001621E8E7042B0DD115210822694468467C
:1036800005F00CFB0098019902F0E0F905F0AAF9A9
:103690003060C4E7052BC2D1152108226944684671
:1036A00005F0FCFA0098019902F0D0F905F09AF9BA
:1036B00030606A7D0A231E21C5E78D5CA018057164
:1036C0000132C5E70D0800209008002028250020C1
:1036D0001000002010B5134B04001B78002B01D103
:1036E000FFF7B2FEFFF720FE00200F4A0F49104BF4
:1036F000545058600130106058680028FCD00020F9
:1037000018610130906018690028FCD0094B0A4804
:103710001B785B011B185350FFF706FEFFF7EAFD0D
:1037200010BDC0460D080020001000400405000038
:10373000FC1000400C0800200E08002030B589B0B5
:1037400000281EDD03230A6813401AD1042A18D961
:103750000F2011680840062813D109091F2910D924
:1037600001240133990051580020214201D0491011
:10377000C8B26D46591E6854202BF2D16846FFF737
:10378000A9FF002009B030BD10B5002813DD0C687A
:10379000E30710D56410532C0DD8084B1B78002B71
:1037A00001D1FFF751FEFFF7BFFDA123044ADB0063
:1037B000D450FFF79FFD002010BDC0460D0800202B
:1037C0000010004010B500280EDD0C68E3070BD593
:1037D0006410FF2C08D8054B1B78002B01D1FFF794
:1037E00033FE034A034BD450002010BD0D080020C7
:1037F000001000402405000013B5002814DD0C68FB
:10380000E30711D5094B64100093094B0193072C72
:103810000AD8084B1B78002B01D1FFF715FE6B4629
:10382000054A1957054BD150002016BDE2ECF0F4C3
:10383000F8FC00040D080020001000400C050000FA
:1038400070B588B0002820DD0324086804401CD12E
:1038500004281AD90F2302681340042B15D1FEF750
:1038600053FD060005F054FE0500122800D912256C
:103870002A0002210D326846FFF790FD6B465D730A
:10388000A54205DC6846FFF725FF002008B070BDA3
:103890002300325D6B449A730134F1E7F0B50D00FB
:1038A0008BB0012831DD0324086804402DD10428A1
:1038B0002BD90F2302681340042B26D14B68DB075A
:1038C00023D5FEF721FD6E6807007310019305F004
:1038D0001FFE05000E2800D90E252A0001211132F5
:1038E00002A8FFF75BFD6A46127902AB5A7302AA7F
:1038F00073129373019B76141B0ED6731374557455
:10390000A54205DC02A8FFF7E5FE00200BB0F0BDE4
:103910003A5D02A963189A740134F1E730B589B0B1
:10392000002814DD0C68E30711D510226846002139
:10393000FFF734FD6B466A4665105D736846631297
:103940002D0E64149373D4731574FFF7C3FE002017
:1039500009B030BD174B184A5968002903D000211F
:10396000596001319160196900291FD00020186148
:103970008023DB00D3581149012B18D1A923DB0088
:10398000D3585B420B600E490B78032B01D80133EF
:103990000B7003200B490B78013303400B700A496D
:1039A0005B015B180949535001239360704708601D
:1039B000FAE7C046FC100040001000400C00002058
:1039C000940800200C0800200E08002004050000C8
:1039D00010B5034A0E21034800F0B4F810BDC046EC
:1039E00020AB000017AB0000044A05491368C85417
:1039F00001339B059B0D13607047C046B00C00203F
:103A0000B008002070B5114C114A2368834202DCD3
:103A10000023236016E0155C411C2E00FA3E012EA7
:103A200005D899420FDA555C013D1F2D01D90800D8
:103A3000ECE70100151A565C6E5401318B42FADC3A
:103A4000181A206070BD1570FAE7C046BC1000203F
:103A5000BC0C002010B5FEF71DFA064B1A68824216
:103A600001D900221A601B68C31A0348984280419A
:103A7000404210BDAC080020204E000010B5094C9B
:103A8000094A23681268934200D110BD074AD05CEE
:103A9000FEF784FB0028F8D0236801339B059B0DBB
:103AA0002360ECE7B40C0020B00C0020B00800202C
:103AB00010B50400064B074A1B6812689B1ADB43CB
:103AC0009B059B0DA34200DB10BDFFF7D7FFF1E77D
:103AD000B00C0020B40C0020F7B505005668019129
:103AE000B000441C06301700FFF7E2FFFB20FFF791
:103AF0007BFF1C20FFF778FFE8B2FFF775FFE0B20D
:103B00002412FFF771FFE0B2FFF76EFF6B461879E2
:103B1000FFF76AFF0025AE4200DCF7BDAB00FB18E3
:103B20009C680135E0B2FFF75FFF2012C0B2FFF7DB
:103B30005BFF2014C0B2FFF757FF200EFFF754FFC2
:103B4000E9E7000070B5074E3368092B08DC0C2547
:103B50005D43054C0133285164196160A2603360F4
:103B600070BDC046B80C00204C250020F0B587B0D1
:103B700002900C00012803DC1B20FCF7ABFC45E0A5
:103B8000244B08680093830709D1042807D90F2321
:103B900002681340042B02D1FEF7B6FB00901D4BC8
:103BA00060680193830709D1042807D90F230268AD
:103BB0001340042B02D1FEF7A7FB01900027164B00
:103BC0001B680493049BBB42D6DD0C267E43134B3B
:103BD0000099F618306805F089FC051E05D1736858
:103BE000B6680593059B9D4201DB0137EAE7306823
:103BF0000199039605F07AFC0836002808D12100C7
:103C00000298039B083102385B68984707B0F0BD03
:103C10000135E7E787A50000B80C00204C250020FF
:103C200010B5FFF719F8FEF75BFAFEF7CDFBFEF7CC
:103C300003FCFFF7CDFE00F00FFE00F0CFFF10BD3C
:103C4000962210B512010021034805F030F8002239
:103C5000024B1A6010BDC04618120020B0050020AB
:103C6000064B074A1B6812689B1ADB439B059B0D9A
:103C70000122834200DC002210007047B00C0020BB
:103C8000B40C0020F8B505000C0016001F1E0ED164
:103C90000320FFF7E5FF002808D0FA20FFF7A4FE75
:103CA000E8B2FFF7A1FEE0B2FFF79EFEF8BD501D9F
:103CB000FFF7D6FF0028F9D0FB20FFF795FEE8B20A
:103CC000FFF792FEE0B2FFF78FFEF0B2FFF78CFE37
:103CD0003012C0B2FFF788FE3C00E31B9E42E5DDD8
:103CE0002078FFF781FE0134F7E7000070B500246B
:103CF000F0250B4B1B68A34202DCFFF7A1FF70BD50
:103D00002B006343074A9B181A78002A05D059787C
:103D1000002311201A00FFF7B5FF0134E9E7C04680
:103D2000B005002018120020F8B507000024F02587
:103D30002B0063430C4A01349E18B74211D03178EE
:103D400000290BD00133D15C002311201A00FFF7AA
:103D500099FF2A000021300004F0A9FF0A2CE7D1C6
:103D6000F8BD024B1C60F9E718120020B0050020D6
:103D7000F0B50400100001220300FFB00D00134055
:103D800013D06B461A706A4669464310537042124C
:103D90001B0E8A700B7105226B464014C8702900F7
:103DA0002000FFF76FFF7FB0F0BD032606401ED155
:103DB00004281CD90F2201680A40042A29D10223B1
:103DC0006A461370FEF7A0FA070005F0A1FBF8237E
:103DD000FF33984200D91800B04202DC421C6B4607
:103DE000DDE76A460136731EFB5C9355F4E7042851
:103DF00001D0002809D16A460323043813704242D7
:103E000050416B4602225870C9E7002ECBD10428DE
:103E1000C9D90F2102681140052913D16E46013915
:103E20003170F8211209FF3192008A4200DD0A0048
:103E3000934201DB0132D2E76E460133C118C978E3
:103E4000F154F5E70629AED11209642A00D964229B
:103E50006E460521317001369A4202DC05235A4331
:103E6000E8E7012701339900415839420BD0394125
:103E7000012737700F127170B7700F14090EF770A9
:103E800031710536E8E70149F2E7C04619FCFFFF4A
:103E900070B502000024F0210D4E08006043801927
:103EA0004578954203D001340A2CF6D170BDF0223A
:103EB000002104F0FCFE074A1368013BA34200D135
:103EC0001460002329001A001120FFF7DBFEEDE744
:103ED00018120020B005002010B5B2B002236A46C7
:103EE0000400137005F014FBC72800D9C720002375
:103EF000984207DC421C6B46FE211420FFF7C2FEED
:103F000032B010BD694601335A1EA25CCA54EFE7B5
:103F100030B5B3B002236A460500137005F0F8FA15
:103F20000400C72800D9C72400239C420BDC2000D2
:103F30003230FFF7BDFD621C6B46FF211420FFF7F6
:103F4000A1FE33B030BD694601335A1EAA5CCA5483
:103F5000EBE70000F7B5234B06001B68F021009348
:103F60000023009A9A4211DC0024F0231A006243D5
:103F7000019201991C4A55182F78002F12D0013454
:103F80000A2CF3D11948FFF7C3FF29E00A005A436E
:103F9000154882185078B04202D11278002A1FD1F9
:103FA0000133DEE7F0223900280004F080FE02230E
:103FB0000D4A0199EB6053540D4AF1008A58009B59
:103FC0006E70AE70AA602F616F61A34202DC054B78
:103FD00001341C60002331001A001020FFF752FE4C
:103FE000F7BDC046B00500201812002091B00000B7
:103FF000781B002010B5FFF779FEFF24084AE30084
:104000005B429B18074AD35C043B012B03D8E04377
:10401000C0B2FFF79FFF013C002CEFD110BDC0469E
:10402000FC070000781B0020F7B50E00FF247F2559
:1040300001901C4AE300D31A1B4A9A181278062AE8
:1040400001D0032A1DD1FF22D2009B181868836873
:104050002B401C2B15D1C3681A002A40042A10D10A
:1040600002692A40192A0CD11B0A01339B000C302B
:10407000C018FEF749F9070005F04AFA0023B042DC
:1040800009D0013C002CD4D1F7BD019AF95CD25C77
:104090009142F6D101339E42F7DCE043C0B2FFF714
:1040A00059FFEEE7781B0020FC07000070B5050003
:1040B000FF24084AE3005B429B18074AD35CAB42EB
:1040C00003D1E043C0B2FFF745FF013C002CF0D123
:1040D00070BDC046FC070000781B0020F7B5FDF757
:1040E000D9FE514B1A68824201D900221A601A681F
:1040F0004E49821A8A4200D883E01860FDF7D4FE48
:10410000071E00D101370020FDF7C0FF01900020FD
:10411000FDF7D0FF019B0090454C464D002B14D07D
:104120002368002B00D07AE02B682760002B00D199
:1041300071E0414B01261B78002B63D10920FFF76A
:10414000B5FF3E4B1E703C4B1E70009B002B12D0E7
:104150002B68002B0FD123682F60002B1ED0374B0C
:1041600001261B78002B52D10920FFF79FFF334B0C
:104170001E70314B1E702368002B0FD02F4E3278EB
:10418000002A0BD19F4200D227602368FB1A312BF3
:1041900004D90720FFF78AFF012333702B68002B17
:1041A0000FD0254E3278002A0BD1BB4200D92F60A8
:1041B0002B68FF1A312F04D90820FFF777FF01235E
:1041C00033702368002B0CD0019B002B09D11B4EB0
:1041D0003378002B02D10720FFF768FF002323600C
:1041E00033702B68002B0CD0009B002B09D1124C94
:1041F0002378002B02D10820FFF758FF00232B6003
:104200002370F7BD0720FFF751FF0C4B9CE70820F8
:10421000FFF74CFFADE7009B002B9CD1ABE7009A6A
:10422000002A95D1AAE7C046A80800200F27000061
:1042300098080020A0080020A40800209C08002066
:1042400037B500240500FFF751FD01A80194FDF7E3
:104250000BFF21002000FEF7EBF9FEF7ABFBFDF7AB
:104260003DFFFDF73CFFFEF7F1FCFDF739FEA542EF
:1042700004D0FDF7A9FF0248FFF74AFE37BDC0464C
:1042800082B00000002310B501001A001120FFF7D2
:10429000F9FC10BD07B56B46197069465A701312C8
:1042A0008B701314120ECB700A716B46010005223D
:1042B0001320FFF7E7FC07BD10B50A00010012202C
:1042C000FFF756FD10BD70B5050008000C00323038
:1042D000FFF7EEFB2B00220000211B20FFF7D2FC92
:1042E00070BD10B50C000300110014202200FFF770
:1042F000C9FC10BD012370B5FF24084A41185B4278
:10430000884201D3D84370BD06781D0A234073400C
:104310009B009B5801306B40F2E7C04664AC000044
:10432000002313B501930B4BC2000400D0580028A2
:1043300005D0436808309900FFF7DCFF01900920A1
:10434000FFF7B6FB01AB042221001720FFF79AFC10
:1043500013BDC046781B002070B506000020FEF794
:1043600017FD0024FF25002801D1200070BD03683F
:104370001A142A40152A07D11B122B40B34200D130
:104380000400FEF705FDEEE71D2AFAD10024F8E748
:10439000F0B580279DB0FFF771FBAD4CAD4D2068A7
:1043A000FF00391A4019FDF7DFFE23680600C31825
:1043B0002360002B0ED11DB0F0BD2068391A2818DB
:1043C000FDF7D2FE236806001B182360FDF762FD8F
:1043D000A14B1860002EF0DC2B78FA2B00D013E1F3
:1043E0002368022B07DCFFF735FB0028E3D0012010
:1043F000FFF708FBDFE76878AC78023818281FD889
:1044000002F0A0FD0D2024282B341E3E6872768C0D
:10441000DEEF1E1E1E1E1E1E1E1E1E1EFD00FF2C7B
:104420000ED02000FFF734FD00228C4BE100CA5073
:104430005B181A712100009213001320FEF7ACFEE6
:104440000320D5E72000FFF785FDF9E72000FFF7FF
:104450001FFDF5E7FFF7CEFDF2E7FFF747FC002071
:10446000FFF7EEFE7E48FFF753FDE9E7632CE7D840
:104470007C4BA200D25821001520FFF779FCDFE722
:1044800000242000FFF768FF061E03D10134642CCE
:10449000F7D1D5E7083005F03BF805000530FFF708
:1044A00007FBFB20FFF7A0FA1D20FFF79DFAE0B203
:1044B000FFF79AFAE8B2FFF797FA2812C0B2FFF7AF
:1044C00093FA3700BB1B9D42E0DD387AFFF78CFA88
:1044D0000137F7E700211D2000910B000A00FEF7CD
:1044E0005BFEFDF771FEABE72000FFF719FFA7E7C2
:1044F000FDF7E2FC03AC5C4A642100905B4B2000BA
:1045000004F0A2FF02232000237005F001F823002D
:10451000020000211620FFF7B5FB91E700244F4A67
:10452000E300D558002D28D06B689E00701DFFF762
:10453000BFFA2B0000253200083321000120FFF7CD
:10454000A1FB0020FEF724FC2F002E00002818D12C
:10455000002F04D03A0001212000FFF7BDFA002D02
:1045600004D02A0002212000FFF7B6FA002E04D062
:10457000320000212000FFF7AFFA0134FF2CCED12A
:104580005EE7FF2103681A120A40A24209D11A14F9
:104590000A400B2A08D10B400CD0012B0CD0022B67
:1045A0000CD0FEF7F5FBD1E7132AFAD100252F0036
:1045B0002E00F6E70600F4E70700F2E70500F0E753
:1045C0000024FFF793FB2200210000942300DA204F
:1045D000FEF7E2FDFF222100D200204804F067FB35
:1045E0007FE7012C02D1FEF7F5FC29E7022C02D16E
:1045F000FEF734FE24E70120FFF722FE20E7002328
:1046000021001A001A2086E7FB2B00D0EFE6226873
:10461000042A00DCE7E62E79E878154B36020643DB
:104620009E4200DDE3E6331D9A4200DCDBE6EB5CF4
:10463000FE2B00D0DBE66B78AC78711E1B2B6BD0A9
:1046400018D8012B2BD0082B3DD0701DD0E6C046CA
:10465000BC100020BC0C0020AC080020781B0020FF
:1046600064B00000702300207BB0000076B0000032
:10467000F60300001D2B60D052D31E2BE5D1012C78
:10468000E3D10029E1DD6B79002B03D01C00322B34
:1046900000DD322464235C43344B1C60D5E7FF2CDF
:1046A000D3D02000FFF7F4FB6D79314AB31E00929E
:1046B00021002A000A20FEF76FFD2E4BE400E05097
:1046C0001B191D71C1E7632CBFD86A79022A13D068
:1046D000032A1BD0012AB8D1E979AB790902194321
:1046E0002B7AA4001B0419436B7A1B060B435B0057
:1046F0001343214AA350A8E70029A6DDB11E1C4898
:10470000FDF7E6FD1C4BA400E0509EE7AB79A4004A
:104710005A1E93419B00ECE71848FFF785FC94E78D
:10472000FF2C92D06A79022A8FD811490B20009170
:104730002100B31EFEF730FD87E70B00632900DD83
:104740006323002203A893420ADCD9430022C9173D
:10475000194041180A700133009021001520E9E743
:10476000A918497981540132EDE7C04604000020C0
:10477000C20C0020781B002070230020C10C0020F8
:104780000122094B1A60094A1368002BFCD003224E
:10479000074B1B68D8171040C0180123801006383B
:1047A000400018437047C04600C0004000C10040B0
:1047B00008C500400120704710B5064C200000F0ED
:1047C00045FB0549200000F069FB0122034B1A60FC
:1047D00010BDC046E8100020801A0600C01000205E
:1047E00010B501210D20FDF76DFB01210E20FDF715
:1047F00069FB00210F20FDF765FB044C200000F051
:1048000061FA1021200000F079FA10BDC8100020D4
:1048100010B504680D20E30703D56410FF2C03D9FD
:104820001720FBF757FE10BDFFF7DAFFE1B2024891
:1048300000F086FA0020F6E7C810002010B5FFF758
:10484000CFFF0021034800F07BFA4300012018430A
:1048500010BDC046C810002010B5034A0721034808
:10486000FFF770F910BDC046A8B00000E0B000002E
:104870000D4B70B51B6804000E001500002B01D114
:10488000FFF79AFFE1B2094C200000F09EFBF1B265
:10489000200000F0A1FAE9B2200000F09DFA20000B
:1048A00000F0FEFB70BDC046C0100020E8100020E4
:1048B00010B501240368234205D04168214202D08B
:1048C0008268224203D10D20FBF704FE10BD581070
:1048D000802801D91520F7E74910FF2901D91620B2
:1048E000F2E75210FF2A01D91720EDE7FFF7C0FFCA
:1048F0000020EBE7F7B501242300A0421BDD0D6883
:104900002C4218D01A4B25411B684C68002B01D152
:10491000FFF752FF0127174EE9B2300000F055FBB8
:104920003C420AD03C413000E1B200F055FA300080
:1049300000F0B6FB00231800FEBD03252540F6D18C
:10494000042CF4D90F2322681340062BEFD113094E
:104950000193019B9D42EADA0135AB00E1583942EF
:10496000F7D04910C9B2300000F036FAF1E7C0467E
:10497000C0100020E8100020144B70B51B68050023
:104980000E00002B01D1FFF717FF114CEDB22900EB
:10499000200000F01AFBF1B2200000F01DFA002107
:1049A000200000F01DFB002801D0404270BD012214
:1049B0002900200000F004FB200000F0FEF9002890
:1049C000FAD0200000F0FEF9F0E7C046C010002049
:1049D000E810002010B501240368234202D041688A
:1049E000214203D10D20FBF775FD10BD5810802822
:1049F00001D91520F7E74910FF2901D91620F2E760
:104A0000FFF7BAFF40002043EFE70000002370B536
:104A1000344D0400EB5601330BD10D211D20FFF75F
:104A2000ABFF5A2814D101222A212A703D38FFF702
:104A30001FFF0023EB56022B2AD0032B49D0012B5A
:104A40004CD121001D200124FFF796FF644225E090
:104A50000F211920FFF790FF332805D102235F2291
:104A60002B7020211A38E2E70D211E20FFF784FF6A
:104A7000C7280AD1032300222A21A9382B70FFF767
:104A8000F7FE1B222A211E20D1E700232B70D0E73E
:104A9000012C13D129211920FFF76EFF7F2801DD9A
:104AA0000138FF3803007F3301DA7F20404264235E
:104AB0007F21584302F0DAFA604370BD032C0BD11A
:104AC0002B211920FFF758FF043CE7E72D2119207F
:104AD000B9E721001E20B6E7052CF7D001240020FD
:104AE0006442E4E71400002010B50120FFF78EFFB8
:104AF00043000120184310BD10B50320FFF786FFC7
:104B000043000120184310BD10B50520FFF77EFFBC
:104B100043000120184310BDF8B50123020018001E
:104B20009A4236DD0E68334233D003244D682C4060
:104B30002FD1042D2DD90F2229680A40062A28D109
:104B4000144B1B68002B01D1FFF736FEEB0704D492
:104B50002B681C09202C00DD20247610F1B20E4EAB
:104B60002200300000F02CFA0435A700EF19AF4204
:104B70000CD0300000F021F90028FAD0300000F00D
:104B800021F901234000184301C5F0E7012064002A
:104B90002043F8BDC0100020E8100020002070471E
:104BA00001207047002070470020704701207047A7
:104BB0000020704700207047002070470020704799
:104BC0000020704700207047002070470020704789
:104BD00000207047704770477047000010B5034AC7
:104BE0000E210348FEF7AEFF10BDC04624B1000001
:104BF00094B1000010B5FDF77FFA0648FDF708FBF9
:104C0000FFF70EF80448FFF783F9FEF72BFBFFF7D9
:104C1000F1F910BDE20400001DB2000010B5FDF76F
:104C2000D3F810BD70B5002504AC24780573A942F3
:104C300005D10A4B0A4A23210A4803F0B3FF016059
:104C40000949920052589B0002715B58A40083717D
:104C50006358856043710223C37170BD35B2000093
:104C60009AB2000043B20000F8B20000037B002BB0
:104C700004D14373837303610133037370470000EE
:104C80001FB50191A02100240068C900D2B2445090
:104C9000012A10D0A24209D0032A0AD0074A835021
:104CA000074B019AC250012343501FBD02221343F8
:104CB000F4E70422FBE70622F9E7C04654050000AA
:104CC0002405000010B50400FFF7D0FFA1222368DF
:104CD000A179D20099506179064A20009950217932
:104CE00004329950044B19685A689B68FFF7C8FF53
:104CF00010BDC0460C050000DC1000204BB2002B9C
:104D00000FDB80233F290FD81F290FD80F290FD879
:104D100007290FD803290FD81B060168074A8B50B3
:104D2000704780239B04F8E7DB04F6E71B05F4E7F4
:104D30005B05F2E79B05F0E7DB05EEE724050000E5
:104D40000368074A99501A00FC32D1680029FCD048
:104D5000A321C90058580023C0B2D3607047C04691
:104D60001C05000007B58022074BD2051A600022FF
:104D70009A6002321A710F230C3200930349023BEE
:104D80000348FFF74FFF07BDDC1000200030004054
:104D9000C8100020F8B505000E0017000024BC4222
:104DA00008D02B68315D1B6828009847002801D087
:104DB0000134F4E72000F8BD704710B51C3000F056
:104DC000A9F910BD10B51C3000F096F910BD10B552
:104DD0001C3000F0A5F910BD70B5437E0D00002B0E
:104DE00001D1002070BD6430040000F0A2F9002859
:104DF000F7D12000290000F070F90120F2E700004F
:104E0000F7B50193FA23002504009B0083600D4B46
:104E10004560083303601C300F00160000F052F9A3
:104E20002000643000F04EF9074A2761B600B358FD
:104E300020006375019B9B009B586576A576A37542
:104E4000FEBDC046D8B20000F8B200000123A02287
:104E5000C375837D0E49C133FF33D2059B00995042
:104E6000437DC133FF339B009950CC220169094B2C
:104E70005204CA5005220169243BCA50827D01694F
:104E80000833CA500269417D034BD1507047C04678
:104E90000C060000240500000C050000A0220023E1
:104EA00010B50469D200A3500A4CA1420FD90A4C94
:104EB0008C425B4109495B420B40CD21C9045B1820
:104EC00004690749635005210369995010BDCC233B
:104ED0005B04F5E7A086010090D00300000098FD78
:104EE00024050000F7B5040000200D000193824264
:104EF00065D01600402A00D9402627001C3738000C
:104F000000F0F6F8B1232269DB00D550802201239E
:104F1000216992008B50A27E002A03D1226913627C
:104F2000226913600025731EAB4207D1019B002B41
:104F300004D0802202212369920099500122236922
:104F40001A622369FC33DA68002A02D19A6A002ABD
:104F5000F9D09A6A002A0BD1DA60A3232269DB0018
:104F6000D1583800C9B2013500F0B7F8B542DAD3EC
:104F7000019B2269002B0FD11300FC339B6A002B8D
:104F80000AD10133A376D3612369FC33DA6C002A9A
:104F9000FCD00022DA640AE000230121A3765161EB
:104FA0001A002369FC3399680029FCD09A602369B0
:104FB000FC339A6A002A01D000229A62E8B2FEBD50
:104FC00010B50123FFF78EFF10BD0300AC3310B501
:104FD00004001970643000F08BF80123637610BD73
:104FE0000023020070B5AC3243760D001178B12277
:104FF00004000069D20081508022216992008B5008
:1050000022690133136222699360260064363000FE
:1050100000F080F8002812D0300000F06DF81E4B30
:105020002269D0502369FC331A6A002A02D19A6A95
:10503000002AF9D09A6A002A01D11A62E5E72369A9
:105040000122002D0DD11900FC31896A002908D1F7
:10505000DA612369FC33DA6C002AFCD00022DA64BE
:1050600007E05A612369FC339A68002AFCD00022C9
:105070009A6000202369FC339A6A82420BD09862BE
:105080002169064A8B588B501800022B03D0181F39
:10509000431E9841033070BD1C050000C40400008D
:1050A00010B50121FFF79CFF10BD000010B51323C0
:1050B000142202490248FFF7A3FE10BD0040004041
:1050C000E810002010B540220021040003F0EFFD9D
:1050D000002320002364636410BD10B53F24026CDC
:1050E000531C2340446C9C4201D08154036410BD86
:1050F0000023036443647047436C026C934206D000
:105100003F21C25C01330B40436410007047012013
:105110004042FBE7036C406C181A00D540307047E2
:10512000436C026C934201D0C05C70470120404246
:10513000FBE73F22036C406C01331340181A4342D3
:105140005841C0B27047000003210A4802680A4370
:105150000260094802680A4302600849084A094B8C
:105160009B1A03DD043BC858D050FBDC00F012F85A
:10517000FAF7CAFF240500405405004004B80000B7
:105180000000002048020020FEE7FEE7FEE7FEE701
:10519000FEE7FEE72D4B10B51A68D2B2012A0FD1F7
:1051A0002B4A126812070BD12A4AE0241168F02218
:1051B0000800104021422DD12749096811422CD006
:1051C0001A68D2B2012A12D12149096809070ED101
:1051D000F020204909680140402908D11E4909688A
:1051E000014204D18020C121C005C90042501B6882
:1051F000DBB2012B0DD1164B1B681B0709D1154BD8
:105200001A68F0231A40A02A0FD1134A12681A42D2
:105210000ED010BD3028CFD0D2E7104A104911600F
:105220008021104A09021160CAE7D02AF1D1ECE7C7
:105230000D4B1A68012A04D00C4A1A601A68012A18
:10524000FCD1C0220A4B1A60E3E7C046E00F00F031
:10525000E40F00F0E80F00F0EC0F00F00405004050
:10526000DFFF07C0186C004000EC0640759300009B
:1052700014EC06400120704710B503681322DB6967
:10528000984710BD70470000054B0269D150036973
:10529000FC331A6A002AFCD0002201201A627047EF
:1052A0001C050000030010B55C331A781F231A4058
:1052B0001E3B19009140114AD167C22204210469A2
:1052C0009200A150026953600269D360A0230022BA
:1052D0000169DB00CA5001230169094A5B428B5016
:1052E0000169084A8B5001690C3A8B5001690832F8
:1052F0008B501430FFF7FCFE10BDC04604E100E007
:105300000C0500001405000010B51430FFF702FF73
:1053100010BD10B51430FFF703FF10BD10B51430E9
:10532000FFF7EAFE10BD0000030070B55E331A7887
:105330000469724BE25003005D331A780469704BC4
:10534000E250030061331C7802696E4B012C00D0DF
:105350009EE005005F352E78A225ED005651020033
:1053600060321578A1220669D200B5500269D45086
:105370009623DB00994200D88CE096231B019942CA
:1053800000D88AE096235B01994200D888E09623F2
:105390009B01994200D885E0E1239B01994200D806
:1053A00082E09623DB01994200D880E0E123DB0113
:1053B000994200D87DE096231B02994200D87AE0FA
:1053C000E1231B02994200D877E096235B029942C1
:1053D00000D874E0E1235B02994200D871E0E12338
:1053E0009B02994200D86EE0474B994200D86CE08E
:1053F000E123DB02994200D86AE0E1220023120394
:105400008A425B41414A5B421340802252059B180D
:1054100001693F4A8B50A02304220169DB00CA5076
:1054200000210369FC33D9600369FC33196201234D
:1054300001690B6001698B60C121046989006250B8
:105440001F215C3002780A4093406231314AFF31BB
:1054500053500021415600293CDA0F230B40083BF2
:105460002D4C9B089B001B1903242140A140FC34B8
:105470008C40DD69A5432C00C0258D4029002143C7
:10548000D9611F23017819401E3B8B40136070BD0A
:1054900000246CE79E23DB02BAE79D231B03B7E7DA
:1054A0001E4BB5E71E4BB3E7EC239B03B0E71D4B48
:1054B000AEE71D4BACE71D4BAAE71D4BA8E71D4B04
:1054C000A6E71D4BA4E71D4BA2E78023DB049FE763
:1054D0001B4B9DE78C080F4BA400E41803230B40E3
:1054E000FF21C025DB009940AD0066598E43310095
:1054F000C0269E4033000B436351C2E70C050000F9
:10550000140500006C05000090D0030000D0BEFE22
:105510002405000000E100E000ED00E000B0130011
:105520000050270000A04E0000F0750000509D00C4
:1055300000F0EB0000903A0100E0D70100B0AF03AB
:1055400000705F07F7B5009308AB1B780025019347
:10555000FA2304009B0083600E4B45600833036010
:1055600014300F001600FFF7ADFD23005C332761F8
:105570001E70009B084A9B00995823005D331970E8
:10558000019B20009B009A5823005E33DD701A7047
:10559000FEBDC0467CB30000F8B20000036910B540
:1055A0001A00FC32D2680400002A0AD0A322D200DA
:1055B00099581430C9B2FFF790FD00222369FC33DB
:1055C000DA6010BD10B50248FFF7E8FF10BDC04615
:1055D000A0110020162307B5022200930249013BC7
:1055E0000248FFF7AFFF07BD00200040A0110020D8
:1055F00010B5002801D003F0BFFE10BD70470000B9
:1056000010B500F011F8FFF7F9FF012000F000FAE3
:10561000FFF7F0FAFFF702FB024B002BFAD000E095
:1056200000BFF7E700000000C420114B80001A58AB
:1056300010491140C02212020A431A50C021802290
:10564000490092025A501A608023A3220021DB05F0
:10565000D20099500122F9309A60074BFF3019505F
:10566000C120023180001950403019501A60704733
:1056700000E100E0FF00FFFF00100140014B186057
:105680007047C04660000020F7B5002320285AD894
:10569000384B8000C258042A5BD007D8022A54D065
:1056A00055D80423012A09D000234CE0062A54D0FF
:1056B00051D31A2A53D002231B2AF5D12E4A11683E
:1056C00008294ED909294FD00A240226A0200125F5
:1056D0002A4AC00015502A482A4D07681C20BF00DE
:1056E00007402948019700685759009027481B0236
:1056F00007401F43C02300989B020340FF205751DF
:105700005759000207401F43019B1F43009B58014C
:105710006023184007433E43565101251C4B15603A
:1057200058680028FCD000205860A1230125DB0028
:10573000D3585560A025ED0050511BB2A14202D0B4
:1057400015D2611ACB401800FEBD0823B6E710231E
:10575000B4E72023B2E74023B0E78023AEE701237C
:10576000ACE708240026B1E70C000126AEE7091BD0
:105770008B40E8E7F8B200005C00002000700040B9
:1057800018000020040500001C000020FF00FFFF9F
:10579000FC700040F0B520285BD8364B8000C25822
:1057A000354B1E68002E30D1C227344BBF00D8596C
:1057B000334C03250440C02000022043D851C024AC
:1057C00080206400800018512E4F18602E4B803CC2
:1057D000D859FF3CA043D8510437D859A843204397
:1057E000D8510837D8590C35A84384460720654658
:1057F0002843D851A820C0001E50C1208026800018
:1058000076021E501C601C4B1C60142500202B00CF
:105810001E4C2E0046433659771C1BD14343E250A1
:10582000A0230325C132FF329200DB05D550184B6F
:105830001A68082A14D114234343E3189A681248BB
:105840005132FF32920059601150DA68C1239B0037
:10585000C250F0BD9642E1D001300328D9D1F8E71B
:10586000082A02D9083AD140E5E708239A1A91405C
:10587000E1E7C046F8B200000412002000E100E0B9
:10588000FF00FFFF04050000009000402000002002
:10589000600000202149F0B54A6C2148002A14D04C
:1058A000A025A12600230124ED05F600C258571CAF
:1058B00006D0C7187F68002F02D027009740AF514D
:1058C00014333C2BF2D100234B64A0230121DB05D0
:1058D00000260F009C4614234B43C3181A1F12685E
:1058E000104C0E4D920014195219526C002A10D00F
:1058F0001A00143A1268551C09D0103B1B68FF2B84
:1059000005D03B00934065461A00074BEA50FC3433
:10591000666401310429DED1F0BDC046FC90004030
:1059200020000020009000400C05000000B5202859
:1059300010D80C4A8000835803290BD8A0220800F5
:10594000C133FF33D2059B0001F0FCFA02090507C1
:105950000021D15000BD0C21FBE70421F9E7032110
:10596000F7E7C046F8B2000020280AD8074B8000AD
:10597000C25801239340A022D205002902D1044934
:1059800053507047A121C900FAE7C046F8B20000A1
:105990000C05000003000020202B0AD8A021A22221
:1059A000C905D2008858034A9B009B58D840012360
:1059B00018407047F8B20000F7B506000D000C0063
:1059C0008B180193019B671B9C4207D03368217899
:1059D0001B683000984701340028F3D13800FEBD21
:1059E0000849094A094B10B51B688858FA22190A58
:1059F0001B0618439200002301F070FC4904C00B01
:105A0000084310BD001001400405000008120020EA
:105A100070B5041E09D0FFF7E3FF050000F014F88D
:105A2000FFF7DEFF401BA042F8D370BD0022044BFD
:105A30009A60044A13680133DBB213607047C046B2
:105A4000FC1001400812002070470000F0B5C64667
:105A500000B5CB0F9846404A4B005B0D9A1882B0B8
:105A60000D000400132A2FDC002A49DB3B4F1741AD
:105A70003E000E40064323D07F08390029400C43E6
:105A80000AD03749BD438C4663445C425C41802365
:105A9000DB021341E4071D434146CE0031492B0090
:105AA0008E192200346875682000290001F0BCFDC1
:105AB000009001910098019922002B0002F04AFC0D
:105AC00002B004BC9046F0BD332A08DD8023DB0021
:105AD0009A42F5D102000B0001F0A6FDF0E7224A40
:105AE0009446012263445242DA400242E8D052080E
:105AF0000242D1D094438022D2051A411443CBE70D
:105B00004B005B080343DBD00B031B0B1C436342BE
:105B1000234380244D0C24031B0B23406D042B4393
:105B200019004346DA000F4B9B181C685D680200A1
:105B30000B002000290001F077FD009001910098F2
:105B4000019922002B0002F005FC42464B005B0845
:105B5000D60733431900B3E701FCFFFFFFFF0F0037
:105B6000EEFBFFFFB0B30000EDFBFFFFF8B5274AE7
:105B70004B005B0D9A180C000700132A10DC002A5A
:105B800036DB234B13410B423AD0802424031441CB
:105B9000002064189C430600250030002900F8BD51
:105BA000332A0EDD80230600DB000D009A42F4D17B
:105BB00002000B003800210001F036FD06000D0048
:105BC000EBE7144D0600AC46012563446D42DD4011
:105BD000AC4663460D000342DFD033239A1A323BB2
:105BE00093401818874200D94C1C63469843D2E76B
:105BF000C90FCC070020531CCDD1074B1C43CAE76B
:105C000006000D000028C0D1C7E7C04601FCFFFF19
:105C1000FFFF0F00EDFBFFFF0000F03F30B5214A12
:105C20004B0087B05B0893421EDD1F4A934205DD9F
:105C300002000B0002F08EFB07B030BD02AA00F09C
:105C400035F803231840049A059B012813D0022835
:105C50001DD0002814D00298039900F037FA802351
:105C60001B069C466144E7E70023002200930023C3
:105C700000F0A6FFE0E70298039900F027FADBE7BF
:105C8000012402980399009400F09AFFD4E70124BC
:105C900002980399009400F093FF80231B069C4612
:105CA0006144C9E7FB21E93FFFFFEF7FF0B54E46B6
:105CB0004546DE465746E0B5E14B4C008FB0904676
:105CC000894664089C4200DC87E0DE4B9C4222DC73
:105CD000DD4A002900DC92E0DC4B02F03BFBDB4BB1
:105CE00006000F009C4200D17EE1D94AD94B02F058
:105CF00031FB02000B00414630000A604B60390066
:105D000002F028FBD34BD24A02F024FB4346012584
:105D10009860D9606BE0D04B9C4200DC8FE0CF4BA9
:105D20009C4200DD55E1CE4A231592469A445146E5
:105D30000905631A19001D00040002F053FE02F069
:105D400087FE02000B00200029000892099302F050
:105D500001FB0022C34B02F08BF80F00060002F09B
:105D600041FE02F075FE04000D0002000B00300041
:105D700039000A940B9502F0EDFA0022B94B02F0BB
:105D800077F8002200230C900D9101F079FA002899
:105D900000D192E1002300222000290001F070FAD6
:105DA000434243410133B04A41460192022208A8CE
:105DB0000092524600F0A4FA4B460500002B16DA7A
:105DC000802243461206944642465B68454263443D
:105DD0005360D3686344D36009E00B00020041467E
:105DE0000A604B600022002300258A60CB602800F7
:105DF0000FB03CBC90469946A246AB46F0BD934BD3
:105E000001F012FC914B06000F009C4200D13DE1D5
:105E10008F4A904B01F008FC02000B004146300015
:105E20000A604B60390002F095FA894A894B01F00B
:105E3000FBFB012543466D429860D960D7E700F02F
:105E400071FF8A4A8A4B06000F0002F011F8002207
:105E5000884B01F0E9FB02F0C5FD050002F0F8FDFA
:105E6000794A7A4B0490059102F002F802000B0087
:105E70003000390002F06EFA754A06000F000498EF
:105E80000599744B01F0F4FF029003911F2D00DC83
:105E9000C7E0029A039B3000390002F05BFA8346A8
:105EA0008A4653465B0024155B0DE31A102B6CDD0C
:105EB00004980599D322674B520501F0D9FF0200DF
:105EC0000B00300039000292039302F043FA0A00FB
:105ED000010013000691079202003900300002F021
:105EE00039FA029A039B02F035FA06000F00049873
:105EF0000599614A614B01F0BBFF32003B0002F0A3
:105F000029FA069E079F0B0002003900300002921A
:105F1000039302F01FFA4B005B0D83468A46E41A96
:105F2000312C32DD04980599B822544B920501F0CA
:105F30009FFF03000C000200029303940B000698DD
:105F4000079902F007FA02000B0006000F000698FE
:105F5000079902F0FFF9029A039B02F0FBF9484A05
:105F60000290039104980599464B01F081FF029A33
:105F7000039B02F0EFF902000B003000390002929F
:105F8000039302F0E7F983468A465A465346414650
:105F900030000A604B60390002F0DCF9029A039B82
:105FA00002F0D8F944460B000200A260E3604B46C1
:105FB000002B00DB1BE75B46236080231B0653445A
:105FC000636080231B069C466144A060E1606D42D3
:105FD0000DE70B00020002F0BDF943460025986072
:105FE000D9601860596002E7D3221A4B520502F0BB
:105FF000B1F9214A214B0D00040002F0ABF9020077
:106000000B00414620000A604B60290002F0A2F913
:106010001A4B194A02F09EF9434601259860D9604F
:10602000E5E602000B003000390002F093F96B1E28
:10603000154A9B009B5883468A46A342A5D130E768
:10604000FB21E93F7BD9024000004054FB21F93F8E
:106050003163621A61B4D03DFB213941FFFFEF7F0C
:10606000EAFBFFFF0000704140B4000083C8C96D27
:10607000305FE43F0000E03F7370032E8A19A33BBA
:10608000C14920259A837B39C0B30000D3220C4B31
:10609000520501F0C9FA0B4A0B4B04000D0001F048
:1060A000C3FA02000B00414620000A604B60290041
:1060B00002F050F9034A044BB9E6032373E6C046E5
:1060C00061B4D03D7370032E8A19A33BF0B54746E7
:1060D000CE4680B587B000920193754B4F00814644
:1060E00088467F089F4263DC02F07CFC002800D1D8
:1060F000D4E04A4643464846414601F0B9FE040012
:106100000D006C4A6C4B01F0B3FE6C4A6C4B01F015
:106110008BFA22002B0001F0ABFE6A4A6A4B02F0B8
:1061200019F922002B0001F0A3FE684A684B01F028
:106130007BFA22002B0001F09BFE664A664B02F0C0
:1061400009F922002B0001F093FE644A644B01F030
:106150006BFA22002B0001F08BFE029003910022CB
:10616000604B2000290001F083FE029A039B060089
:106170000F002000290001F07BFE009A019B040023
:106180000D004846414601F073FE02000B0020005E
:10619000290002F0DFF802000B003000390002F0A5
:1061A000D9F802000B0000204F4902F0D3F870E04C
:1061B00002000B0001F05CFE04000D003D4A3E4B66
:1061C00001F056FE3D4A3E4B01F02EFA22002B0014
:1061D00001F04EFE3B4A3C4B02F0BCF822002B0083
:1061E00001F046FE394A3A4B01F01EFA22002B001C
:1061F00001F03EFE374A384B02F0ACF822002B008B
:1062000001F036FE354A364B01F00EFA2B00220023
:1062100001F02EFE354B029003919F429FDD344BDF
:1062200000229F423DDC334900207B182E49160096
:106230001F0002F08FF8049005910022294B2000E6
:10624000290001F015FE32003B0002F083F8029AAB
:10625000039B06000F002000290001F009FE009AB0
:10626000019B04000D004846414601F001FE02007A
:106270000B002000290002F06DF802000B00300036
:10628000390002F067F802000B000498059902F04B
:1062900061F807B00CBC90469946F0BD0020124949
:1062A000F7E7154B002604920593144FC5E7C04647
:1062B000FFFF3F3ED43888BEE9FAA8BDC4B1B4BDE3
:1062C0009EEE213EAD529C804F7E923E9015CB19A2
:1062D000A001FA3E7751C1166CC1563F4C55555539
:1062E0005555A53F0000E03F0000F03F3233D33F5B
:1062F0000000E93F0000E0FF0000E73F0000D23F60
:10630000F0B5DE464E4645465746E0B5DC4CA54462
:106310000D9114001900A49A0993DA4B9200D658F3
:106320004D1E03901821E01E0696029500F09EFE79
:10633000C3430100DB1719404B1C9A009B1ADB007A
:106340001B190B9105934C1B771918D4A59BA5001D
:106350009C463F1922AE6544013707E0286802F0E9
:1063600077FB013403C60435BC4208D0002CF5DAB3
:1063700000200021013403C60435BC42F6D1069B3F
:10638000002B01DA00F0FDFB069B03990133DB00D3
:106390009A46099BDA00944600920022914672AA1E
:1063A0000492B94A6144934688469AAB63449B443D
:1063B000029B002B00DABCE15D4600260027039C0F
:1063C0004D442A686B6803CC01F052FD02000B00BB
:1063D0003000390001F028F9083D06000F0044455F
:1063E000EFD1049B4B441E605F6008239C46E14450
:1063F000D145DDD10EA804218446494261448C4632
:10640000069A93009C44614684460A910399083B8E
:1064100063448C460C93009B009263449B46009A15
:106420000498D10003008C46634408911E685F689D
:10643000002A33DD954980468C466244D300984457
:1064400070AB9A460EAB99460022914B3000390052
:1064500001F00EFD02F0C6FA02F0FAFA00228D4BAE
:1064600004000D0001F004FD02000B0030003900B3
:1064700001F070FF02F0B6FA4B4601C3994643465D
:1064800020001A685B68290001F0CEF808235B42FF
:106490009C46E04406000F00D045D5D1059B300056
:1064A0001A003900984600F0DDFCFF2300229B050E
:1064B00004000D0001F0DCFC00F038FC0022764BFB
:1064C00001F0D6FC02000B002000290001F042FF81
:1064D0000D00040002F086FA814602F0B9FA0200CB
:1064E0000B002000290001F035FF060040460F0098
:1064F000002800DCEEE0009B18215A1E92000EAB33
:106500009B58091A1D000D41A9448D405D1B0EAB1F
:106510009D5017231B1A1D41002D2DDD01239C4684
:10652000009BE144002B00DC1CE20E9C0123002CAC
:1065300000D0B5E0009A012A09D099000EAA54585B
:106540000133002C00D0ACE0009A9A42F5D1059BB3
:10655000002B0EDD012B00D1A8E1022B09D1009BFD
:106560000EA95A1E92000EAB9B5807939B029B0AE2
:106570008B50022D00D1C1E00023002230003900F1
:1065800000F07EFE009B002800D194E2069A591E7E
:106590008A4210DC414A0A9894460EAA6344944603
:1065A00000229B0063441C68043B22438342FAD1CF
:1065B000002A00D0C0E0069B0EAA013B9B00D358E6
:1065C000002B00D0B3E001220C9B043B5968013240
:1065D0000029FAD0009B9C466244110007921A00E1
:1065E00001338B4246DC0B9863468046A59C4344AE
:1065F000A046099C9B00A1464A449844D30022AA85
:106600009146049A99449446089BA59A634484460B
:10661000614494469A468B0063440093434658680D
:1066200002F016FA4B4618605960029B002B24DBDF
:106630004D46039C0026002701E0286869680CCCC1
:1066400001F016FC02000B003000390000F0ECFFF6
:10665000083D06000F005C45EFD153469E60DF60A9
:1066600004239C460433E0449C46009BE144E244FE
:106670009845D3D1079B0093D1E600260027ECE78D
:1066800094FDFFFF88B5000018FEFFFFFFFFFF1F0E
:106690000000703E0000704100002040FFFFFF3FFF
:1066A000002180225204141B0EAA545000999942D2
:1066B0000EDD0EA884469B000EAA8900D2586144C4
:1066C0006344CF4800E01A68821A04C38B42FAD1AF
:1066D00001243CE7059B002B06D1009B0EAA013B41
:1066E0009B00D558ED1517E70022C64B300000F08F
:1066F000EBFD002800D024E100253DE732003B00FF
:106700000020C14901F026FE06000F00002C00D138
:1067100032E7059A0020BC4900F0A4FB02000B0000
:106720003000390001F016FE06000F0024E70122B8
:1067300050E70026002754E64B46059A0793884603
:106740008B000EA9CB58183A08950592002B0DD155
:106750008C464146AD4B43449B006344043B586820
:106760000139183A0028F9D088460592059A002088
:10677000A54900F077FB434604000D00002B00DA2A
:1067800005E29E000EAB9C464346DB0066449C46F9
:10679000059370AB9946049F67440097306802F0F8
:1067A00057F922002B0001F063FB0022386079606A
:1067B000974B2000290001F05BFB083F04000D000F
:1067C000043EB945EAD14AAB03939B4600239A465F
:1067D000069B4246994643460132029204934B4639
:1067E000002B00DAAAE080208A4B009D9846C00565
:1067F000894900260027002408E008239C46083524
:10680000E044544511DC4346186859682A686B68AF
:1068100001F02EFB02000B003000390000F004FFF5
:10682000013406000F00A145E7DA5B46C0C39B4672
:1068300001239C46009BE244083B0093029B9A453F
:10684000CDD1049B9846A49B022B00DD8EE0002B4B
:1068500037DC1FD1059B00271D00039B00249C46AD
:106860001E006544083E2A686B683800210000F06D
:10687000DBFE083D07000C00AE42F4D1089B002B64
:1068800003D080231B069C4664443A0023000D99E4
:106890000A604B600720079B18409B239B009D4488
:1068A0003CBC90469946A246AB46F0BD009B0EA963
:1068B0005A1E92000EAB9B5807935B025B0A8B50EB
:1068C00057E64346002B00DA70E100200021DB0090
:1068D0004AAAD61848AF32687368083E00F0A4FE92
:1068E000B742F8D1089B002B00D025E10B00020035
:1068F0004A984B990D9C2260636001F02BFD434642
:1069000007000C00002B13DD01254CAEB14638000A
:106910002E0021004C4601360CCC00F085FEA1462D
:10692000B045F7DA089B07000C00002B00D015E1FA
:106930003A0023000D998A60CB60ABE70026002760
:1069400073E701239C46009BE1440225002B00DDF8
:10695000EBE532003B0000202B4901F0FBFC060078
:106960000F0009E60024F2E54AAB0393A49B032B36
:1069700000D08FE74346002B00DC14E1039ADB00D4
:106980009B46130091465B441E685F68234B43445B
:106990000293DB00994448AB9A464B465C681B68FF
:1069A0001800210032003B000090019100F03CFEF5
:1069B00004000D0002000B000098019901F0CAFCD0
:1069C0003B00320000F030FE4B469860D9601C60FE
:1069D0005D6008235B429C46E14426002F00CA45C7
:1069E000DBD14346012B00DCE3E0039A13005B4458
:1069F0001E685F68029BDB0099464A44904610E09F
:106A0000FFFFFF000000E03F0000F03FFFFFFF3FFF
:106A10000000703E48B50000FB21F93FFFFFFF1F5B
:106A2000984643465C681B681800210032003B0012
:106A30000090019100F0F8FD04000D0002000B0031
:106A40000098019901F086FC32003B0000F0ECFD5B
:106A50004346039A9860D9601C605D60083B26003D
:106A60002F009A42DCD14D4694460026002447462A
:106A7000083565442A686B683000210000F0D4FDB9
:106A8000083D06000C00AF42F4D1039B4A9F5D68AD
:106A90009968D868089B002B65D08022120694461E
:106AA0000D9B6544604464441F605D609960D860DC
:106AB0001E615C61EEE69A464B460793059B3000EB
:106AC0005A423900089500F0CDF900223A4B0600F1
:106AD0000F0000F0F9FB002824D0384B00223000D2
:106AE000390001F0C5F901F07DFF52460400950020
:106AF00001F0AEFF0022304B01F0BAF902000B00AA
:106B00003000390001F026FC01F06CFF0EAA505154
:106B10000122059B524418339046059393000EAA18
:106B2000D45023E65346300039009C0001F05AFF50
:106B30000EAB1851D04619E680230D9A1B06CB18D0
:106B4000106053600B0002004A984B9901F002FC60
:106B5000434607000C00002B00DDD5E680231B0612
:106B60009C466444E4E62B003A000D9D2A606B606D
:106B70000A000300AA60EB60320023002A616B6107
:106B800088E6099BDB00009372AB049332E4A49B7C
:106B9000022B00DDE8E6002B00DD92E600D079E66E
:106BA000002700246AE6002600246EE7002000216A
:106BB00098E60026340068E7000070410000703E4F
:106BC000F0B5CE46474680B587B000920193474A5C
:106BD0004B00814688465B08934207DC41464846A5
:106BE00001F000FF4146031E484666D04A46434630
:106BF0004846414601F03CF904000D0002000B003C
:106C00004846414601F034F9394A3A4B06000F0034
:106C10002000290001F02CF9374A384B01F09AFB8B
:106C200022002B0001F024F9354A364B00F0FCFC21
:106C300022002B0001F01CF9334A344B01F08AFB8F
:106C400022002B0001F014F9314B324A00F0ECFC29
:106C50000E9B02900391002B34D0009801990022E2
:106C60002D4B01F005F9029A039B04900591300029
:106C7000390001F0FDF802000B000498059901F0BD
:106C800069FB22002B0001F0F3F8009A019B01F050
:106C900061FB224A04000D00214B3000390001F055
:106CA000E7F802000B002000290000F0BDFC020004
:106CB0000B004846414601F04DFB07B00CBC904626
:106CC0009946F0BD02000B002000290001F0D0F829
:106CD000124A134B01F03EFB32003B0001F0C8F8B2
:106CE0004A46434600F0A0FCE7E7C046FFFF3F3EB0
:106CF0007CD5CF5A3AD9E53DEB9C2B8AE6E55A3E46
:106D00007DFEB157E31DC73ED561C119A0012A3FE1
:106D10001111813FA6F810110000E03F495555556B
:106D20005555C53F49004B0819007047474AF0B513
:106D30004F4691464B005B0D99444646D6464A461F
:106D4000C0B505000C000E0088460700132A27DC9A
:106D5000002A4BDB3E4B13419A460B005246134030
:106D6000034318D03B4A3C4B2800210000F05CFC58
:106D70000022002300F09EFA002847D0002C04DAFD
:106D800080234A465B0313419844464653460027F6
:106D90009E43380031001CBC90469946A246F0BD87
:106DA000332A08DD8023DB009945F4D102000B0073
:106DB00000F03AFCEFE7294A94460122634452422C
:106DC000DA4092460242E6D0224A234B28002100B4
:106DD00000F02AFC0022002300F06CFA002815D0F5
:106DE000002C1EDB534646469F430FE0194A1A4BC0
:106DF0002800210000F018FC0022002300F05AFABD
:106E0000002803D0002C04DB0027002638003100C6
:106E1000C1E76400640825430027002DF6D0104E1A
:106E2000F4E74B46142B0BD03422D21A01239340A3
:106E30005D19BD4208D201239C462F00E044D1E7F2
:106E4000133B9C46E044CDE72F00CBE701FCFFFF5E
:106E5000FFFF0F009C7500883CE4377EEDFBFFFFD1
:106E60000000F0BF4B0070B55B0D14000A00002B52
:106E70001AD14B005B08034315D0234B002200F0CE
:106E8000F7FF224B9C422DDB0A004B005B0D363B8B
:106E90001F4DE318AB422ADC002B0DDD1D4C1B05FA
:106EA00022401A43110070BD1B4DAB42F0D10200CD
:106EB0000B0000F0B9FBF6E71D00353519DA174B6A
:106EC00002009C4209DD0B001548164900F032F81B
:106ED000134A144B00F0CCFFE5E70B0012481349AE
:106EE00000F028F8104A114B00F0C2FFDBE7020067
:106EF000E9E7084C363322401B05134319000022F2
:106F00000B4B00F0B5FFCEE700005043B03CFFFF55
:106F1000FE070000FFFF0F80FF07000050C30000C6
:106F20009C7500883CE4377E59F3F8C21F6EA501BA
:106F30000000903C30B54A00DB0FDB0752081A43D3
:106F4000110030BD02B4714649084900095C49008E
:106F50008E4402BC7047C046002243088B4274D363
:106F600003098B425FD3030A8B4244D3030B8B424A
:106F700028D3030C8B420DD3FF22090212BA030C53
:106F80008B4202D31212090265D0030B8B4219D334
:106F900000E0090AC30B8B4201D3CB03C01A524154
:106FA000830B8B4201D38B03C01A5241430B8B429C
:106FB00001D34B03C01A5241030B8B4201D30B0385
:106FC000C01A5241C30A8B4201D3CB02C01A5241AC
:106FD000830A8B4201D38B02C01A5241430A8B426F
:106FE00001D34B02C01A5241030A8B4201D30B0258
:106FF000C01A5241CDD2C3098B4201D3CB01C01A72
:10700000524183098B4201D38B01C01A524143097B
:107010008B4201D34B01C01A524103098B4201D369
:107020000B01C01A5241C3088B4201D3CB00C01AD6
:10703000524183088B4201D38B00C01A524143084E
:107040008B4201D34B00C01A5241411A00D2014673
:10705000524110467047FFE701B5002000F0F0F8FC
:1070600002BDC0460029F7D076E7704703460B43C0
:107070007FD4002243088B4274D303098B425FD331
:10708000030A8B4244D3030B8B4228D3030C8B425D
:107090000DD3FF22090212BA030C8B4202D3121243
:1070A000090265D0030B8B4219D300E0090AC30B18
:1070B0008B4201D3CB03C01A5241830B8B4201D3C5
:1070C0008B03C01A5241430B8B4201D34B03C01AAE
:1070D0005241030B8B4201D30B03C01A5241C30A26
:1070E0008B4201D3CB02C01A5241830A8B4201D397
:1070F0008B02C01A5241430A8B4201D34B02C01A81
:107100005241030A8B4201D30B02C01A5241CDD225
:10711000C3098B4201D3CB01C01A524183098B4270
:1071200001D38B01C01A524143098B4201D34B0159
:10713000C01A524103098B4201D30B01C01A5241BC
:10714000C3088B4201D3CB00C01A524183088B4243
:1071500001D38B00C01A524143088B4201D34B002C
:10716000C01A5241411A00D201465241104670479E
:107170005DE0CA0F00D04942031000D340425340A3
:1071800000229C4603098B422DD3030A8B4212D363
:10719000FC22890112BA030A8B420CD38901921195
:1071A0008B4208D3890192118B4204D389013AD0D2
:1071B000921100E08909C3098B4201D3CB01C01AA7
:1071C000524183098B4201D38B01C01A52414309BA
:1071D0008B4201D34B01C01A524103098B4201D3A8
:1071E0000B01C01A5241C3088B4201D3CB00C01A15
:1071F000524183088B4201D38B00C01A5241D9D22D
:1072000043088B4201D34B00C01A5241411A00D2AD
:107210000146634652415B10104601D34042002BA9
:1072200000D54942704763465B1000D3404201B528
:10723000002000F005F802BD0029F8D016E77047DD
:107240007047C046D0400B1C1141203A03D49C46E5
:107250001341184363465242934018437047C04657
:107260008446101C62468C46191C634600E0C046EA
:107270001FB500F095FD002801D40021C8421FBDB4
:1072800010B500F0EDFC4042013010BD10B500F02B
:1072900087FD002801DB002010BD012010BDC04685
:1072A00010B500F07DFD002801DD002010BD01209B
:1072B00010BDC04610B500F00FFD002801DC002015
:1072C00010BD012010BDC04610B500F005FD00281E
:1072D00001DA002010BD012010BDC046F0B5CE4639
:1072E000474615042D0C2E0080B50704140C3F0CE6
:1072F0009946030C7E435D43674363437F19340C17
:10730000E4199C46A54203D980235B029846C444F5
:107310004B4643435143250C36046544360C240444
:10732000A4195B19591820000CBC90469946F0BD71
:10733000F0B54E4657464546DE46E0B543025B0A89
:10734000450083B00F1C99462D0EC60F002D57D057
:10735000FF2D24D08020DB00C00418430023814689
:107360009A469B467F3D7C027A00FB0F640A120E10
:10737000984623D0FF2A4BD0E30080240020E40469
:107380007F3A1C43AD186B1C474601935346774028
:107390003A000F2B48D87D499B00CB589F46002BC5
:1073A00000D085E008339A46063B9B467C027A0073
:1073B000FB0FFF25640A120E9846DBD1002C00D08B
:1073C00090E0524601231A4392460120DBE74C46E7
:1073D00058461700022824D0032800D1CFE000220D
:1073E000002301284DD15802D205400AFF0710435F
:1073F000384303B03CBC90469946A246AB46F0BD2C
:10740000002B5BD104239A46033B00259B46AAE749
:10741000FF35002C60D1524602231A4392460220C7
:10742000B1E7FF220023DEE74B461B0C9C464B4690
:107430002604360C180461463300220C6446000C06
:1074400043434E435043544380191A0C121896423A
:1074500003D9802149028C4664441B041B0C100490
:10746000C01883015E1EB341800E1843130C1B1914
:107470009B0103431C00230179D5012362081C40B2
:107480001443019A7F32002A4DDD630704D00F2395
:107490002340042B00D00434230103D53C4B019A34
:1074A0001C408032FE2ABCDCA3015B0AD2B29AE700
:1074B0000C239A46093BFF259B4654E7180001F030
:1074C00053FB4A46431F76259A4000236D4291465E
:1074D0002D1A9A469B4646E7524603231A43924684
:1074E000032050E7200001F03FFB431F2D1A9C4072
:1074F000763D002047E780230027DB03FF2272E769
:10750000424666E74C463200584662E780234A46C8
:10751000DB031A4222D01C4220D123435B025B0AC8
:107520004746FF225FE701239A1A1B2A21DC23002A
:107530000199D3409E318C401A0023005C1EA34168
:1075400013435A0704D00F221A40042A00D00433F0
:107550005A0111D49B015B0A002244E780234A466A
:10756000DB0313435B025B0A3700FF223BE7019515
:1075700087E70022002336E70122002333E7802338
:10758000DB0323435B025B0AFF222CE798B5000074
:10759000FFFFFFF770B500283DD0C317C5185D4049
:1075A000C40F280001F0E0FA9E22121A962A07DC86
:1075B000D2B2082833DD083885406802400A23E04B
:1075C000992A0BDD052329001B1AD94003001B3320
:1075D0009D402B005D1EAB4119430D00052801DDC8
:1075E000431F9D402B000F490B406E0709D00F260B
:1075F0003540042D05D004335D0102D59F220B4098
:10760000121A9B01580AD2B24002D205400AE4077E
:107610001043204370BD002400220020F4E76802DC
:10762000400AF1E7FFFFFFFBF0B54F464646D6465E
:107630000C000903C0B5490A470F5E0039431F0318
:10764000DB0F9C4665007B0A570F1F436D0DE40F4F
:10765000760DA146C000B846D200AB1B64457BD076
:10766000002B5FDD002E00D0A4E03E00164300D1C9
:1076700012E15E1E002E00D09EE1871A4346B842FA
:1076800080410125C91A4042091A0B0200D431E198
:1076900049024E0A002E00D16EE1300001F064FA7A
:1076A0000300083B1F2B00DD61E120223900D21AC4
:1076B0009E40D1409F400E439D4200DD51E15D1B45
:1076C0006B1C1F2B00DD7CE12021C91A3D0030001E
:1076D0008F408840DD40791E8F41310007222843CA
:1076E000D940002507433A40002A09D00F233B40E8
:1076F000042B05D03B1DBB42BF417F42C9191F006F
:107700000B0200D426E26A1CC64B55056D0D9A4249
:1077100000D106E1C44AFF080A40530752023B4326
:10772000120B8EE0002B00D0B8E06B1C5B055B0DEC
:10773000012B00DC30E1871A4346B842B641CB1A30
:1077400076429E1B330200D54CE13B003343A1D16E
:1077500000220024002570E0002B00DCE5E0002E74
:1077600000D183E0AF4EB54260D080263604374367
:10777000B846382B00DC3EE1434613431F007A1E17
:1077800097413F1887428041404209180B0200D4BC
:10779000B0E0A44B01359D4200D1C3E0A24A7B0872
:1077A0000A4001210F401F435108D30707221F43FE
:1077B0003A4099E79B4EB54238D08026360437438D
:1077C000B846382B00DDDCE01F2B00DC30E11E006A
:1077D0004746203EF740BC46202B04D04026F31AF3
:1077E00046469E403243170063467A1E97411F4328
:1077F000CCE0002B00D104E24346134300D159E111
:107800004B07C00818438023C9081B03194208D03E
:107810004546ED081D4204D14346D00859070843A8
:107820002900420FC9007F4D1143C0004B07CA0811
:107830007C49C00803438D4268D012036D05120BCA
:107840006D0D002112031800130B0A0D12051A43C7
:10785000764B2D0513402B435B00E4075B08234365
:1078600019001CBC90469946A246F0BD3E00164346
:1078700012D05E1E002E00D000E1871887428041A2
:1078800041444042091801250B0233D5022585E702
:1078900064463300414610001D00C7E7002D00D0AC
:1078A000DAE00C000443F3D05C1C00D19FE15D4C96
:1078B000A64200D12FE1DB43382B00DD66E11F2B10
:1078C00000DD83E120240500E41A0F00DD40D940EB
:1078D000A0404346A7405B1A441EA04198462F4350
:1078E0003843171ABA42924143465242991A6446A3
:1078F0003500CAE607223A40002A00D0F6E64B07D8
:10790000CA084849FF083B438D4296D119001143EC
:1079100000D19EE1802109030A431203120B414D5D
:107920008FE71500002200238BE7002B00D0C7E073
:107930006B1C5F057F0D012F00DCF1E0394DAB4280
:1079400000D1B9E085180A00854289414244494284
:1079500051180722CF076D082F4349083A401D00F0
:10796000C2E607223049ED1A31403A40BCE63E00FB
:107970002838864000279FE6380001F0F5F82030CF
:107980008EE6434613431F007A1E9741C71BB84239
:1079900080414042091A78E60E003B00064313433B
:1079A000002D61D1002E00D0F4E0002B00D11BE1AE
:1079B00064463900100039E71A4FBB427AD03300D1
:1079C000FFE630001F3DE840202B03D04021CB1ABA
:1079D0009E4037437B1E9F41072207433A400021C8
:1079E000002589E7171A4346BA42B641591A76422A
:1079F0008E1B64464EE61F2B00DDADE02026474679
:107A0000F61AB740B9461700B246DF404E463E432D
:107A100037005646B240561EB24117434246DA403E
:107A20008918AEE6FF070000FFFF7FFFFFFF0F8012
:107A300020264746F61AB740B9461700B246DF403F
:107A40004E463E4337005646B240561EB24117439B
:107A50004246DA40891A99E77F4CA6425BD08024DF
:107A600024045B42214327E7002E0CD1002B00D1D8
:107A7000CBE0644639001000774DD7E6764FBB4225
:107A800018D0330075E6002B14D04B07C0081843FC
:107A90008023C9081B03194207D0FC081C4204D1EB
:107AA0007907D0080843E14621004C46420FC9003F
:107AB0001143C000684DB9E61D0000220023C0E656
:107AC000002D5BD10D00054300D1E2E65D1C00D125
:107AD000B0E0614DAE421FD0DB43382B71DC1F2B71
:107AE00000DD96E020250F00ED1AAF40B9460700F3
:107AF000AA46DF404D463D432F005546A840D94099
:107B0000451EA84188440743BF18974292415142FD
:107B1000414435003AE6644635004146100085E6AA
:107B20000B000343002D00D063E6002BF5D0434645
:107B3000134300D17AE687188742804107224144E7
:107B4000404209183A400B0200D4D5E6434B0135B8
:107B50001940C9E5380069E61E004746203EF74057
:107B6000BC46202B04D04026F31A46469E403243A2
:107B7000170063467A1E97411F4302E6364DAE4218
:107B8000CAD080252D045B422943A6E70843411E45
:107B90008841A6E6002B00D148E6871A4346B84242
:107BA000B641CB1A76429E1B33024BD5171A434679
:107BB000BA429241591A5242891A072264463A40FF
:107BC00092E501430F00791E8F419DE71C000F00D5
:107BD000203CE740202B03D04024E31A994008437F
:107BE000411E884138437CE60022002425E6171A0E
:107BF0004346BA429241591A5242891A64463500A4
:107C000043E541461000144D10E680220024120383
:107C100080E61D000F00203DEF40BC46202B03D026
:107C20004025EB1A9940084307006346781E8741B8
:107C30001F4369E7871897429B4141445B42C9183B
:107C40003500A3E53B003343CED0072231003A4054
:107C500052E600231A00F4E5FF070000FFFF7FFF54
:107C6000F0B54F464646D6468446C0B58046194EC6
:107C700018030F034D00000B5C0082463F0B6D0D97
:107C8000C90F9146640DDB0F0120B5420AD0B44202
:107C900003D0A54201D157450CD01CBC9046994653
:107CA000A246F0BD66463E43F7D1AC42F5D15446FC
:107CB0001443F2D10120C845EFD1994207D0002DDD
:107CC000EBD163461F433800471EB841E5E700206B
:107CD000E3E7C046FF070000F0B54F464646D646EC
:107CE0004D00C0B50E03C90F8A462C491F035C0026
:107CF0008046360B6D0D91463F0B640DDB0F8D42B8
:107D00001ED08C4216D0002D1ED130438446002C4C
:107D100001D13A4323D06246002A1AD09A4529D08D
:107D2000514602200139084001381CBC9046994652
:107D3000A246F0BD39001143E5D002204042F4E7ED
:107D40003043FAD1AC420FD0002C0FD13A43E7D0E8
:107D50000CE00122013B934318000130E5E7634644
:107D60000020002BE1D0DBE73A43E6D19A45D7D19A
:107D7000A542D5DCA54205DBBE42D1D808D0002003
:107D8000BE42D2D250460123013898430130CCE79D
:107D9000C845C5D80020C845F4D3C6E7FF07000092
:107DA000F0B54F464646D6464D00C0B50E03C90F46
:107DB0008A462E491F035C008046360B6D0D9146A6
:107DC0003F0B640DDB0F8D4218D08C4211D0002D7B
:107DD00018D130438446002C1ED13A431CD163464F
:107DE0000020002B30D051460220013908400138D4
:107DF0002AE039001143EAD0022025E03043FBD1CC
:107E0000AC4226D0002C26D13A4324D15146022040
:107E100001390840013817E06246002A0FD09A4520
:107E2000E1D1A54205DBBE42DDD819D00020BE421B
:107E30000AD25046012301389843013004E0012260
:107E4000013B9343180001301CBC90469946A24662
:107E5000F0BD3A43D0D19A45C5D1A542C3DCE0E795
:107E6000C845C0D80020C845E3D3EDE7FF070000B0
:107E7000F0B55746DE464E464546E0B58346060019
:107E80000F03480087B092461D003F0B400DCC0FFA
:107E9000002800D16FE0DE4B984238D08023FF00ED
:107EA0001B041F43730F3B430193DA4B0027994692
:107EB00000239B46F60081442B0369001B0B5246AE
:107EC0009846490DED0F002900D185E0D04B99422D
:107ED00000D173E04346DA0080231B04134352466B
:107EE000CC48520F84461343524600206144D200CE
:107EF00089442100694000918C46012149448A4609
:107F00000F2F00D990E0C449BF00CF59BF465B4650
:107F10003B43019300D06AE10223082700268146F3
:107F20009B46C9E732005846019B614600910228F2
:107F300000D175E0032800D1FEE1012800D02CE13A
:107F400000230027002600253F032A0D3F0BB348DE
:107F500012053A4302401B051343009A5B00D10708
:107F60005B080B433000190007B03CBC90469946B3
:107F7000A246AB46F0BD5B463B43019300D12FE1E7
:107F8000002F00D1A5E1380000F0EEFD03000B3B0F
:107F90001C2B00DD96E11D22D31A5A460100DA405F
:107FA0005E4608398F4013008E403B4301939C4B43
:107FB00000271B1A994600239B467DE741465346FE
:107FC0000B4393498C46E144002B00D01AE1022276
:107FD0000220174300228CE7134300D10DE14346F2
:107FE000002B00D181E1404600F0BEFD02000B3ABB
:107FF0001C2A00DD72E10100434608398B40984697
:108000001D239A1A5346D3401A004346134352463F
:108010008A404946081A824989468144002068E717
:108020007B4B002700268EE7140C1204120C110063
:10803000370C3604350C794328008C462E006043FB
:108040006044834656432100300C804658467943AD
:1080500040440291844506D98846802149028C46D5
:10806000E044414602913604010C360C00048B4674
:1080700081191E0C1B041B0C0391190079438C46BB
:10808000280075436544A8465843050C454477438A
:10809000A94203D9802149028C466744290C8C46A9
:1080A00039000004000C2D042D186144AB440591E7
:1080B0005946049101990F043F0C080C39005143B3
:1080C0004243904602008C46090C8B4662437C4337
:1080D00044445C44A04503D9802149028846424477
:1080E000210C884661460904090C8C463900594325
:1080F000434370437E430F0CF6182404BE196444B6
:1081000042448C46B34203D980235B0298464044E4
:10811000029B61469846049B370443449B46AB450B
:10812000AD416B420D0405992D0C8C467F196744B7
:10813000FD18A8465D462D19A542A4419346644208
:10814000A446C344DC448F42BF4198459B419345BC
:108150009241A445A4415B427F421F43360C5242E8
:108160006442BF192243BF18624638184302D20D39
:10817000039913436A020A43501E82416146ED0D82
:108180002A434E023243D90100D4B3E001265008FD
:1081900032400243DE0732435B08224C5444002C39
:1081A00062DD510709D00F201040042805D0101DB2
:1081B0009042924152429B180200D90104D580247A
:1081C0001948E400034054441848844200DD27E77E
:1081D0005E075B02D2081F0B630516435B0DB2E618
:1081E000002399460133042700269B4664E60323B7
:1081F000019781460C279B465EE60122012017432A
:10820000002276E6032303201F43434671E6C0465F
:10821000FF07000001FCFFFFD8B50000FFFF0F8043
:108220000DFCFFFFFF030000FFFFFFFEFE07000045
:108230000023802700933F030026434B83E6019BE6
:108240003200A446584670E6AC466EE68027019997
:108250003F0339422DD03B422BD11F433F033F0BFD
:1082600000951600384B6EE601252D1B382D00DDDC
:1082700066E61F2D40DC35481C0050441600824045
:108280008440EE40501E824134431443EB40620769
:1082900009D00F222240042A05D02200141D944246
:1082A000804140421B181A023ED5012300270026B8
:1082B00049E68027019B3F031F433F033F0B009488
:1082C000214B40E603005A46283B9A400026019283
:1082D0006DE6584600F048FC203057E60300524651
:1082E000283B9A401300002293E6504600F03CFCE5
:1082F00020307BE6CA4650E71F201E004042041B88
:10830000E640202D03D0124C5444A3401A43501E83
:108310008241324307260027164009D00F20002350
:10832000104014000428B9D122005E075B021F0B25
:10833000D2081643002306E680273F031F433F036E
:108340003F0B1600004BFEE5FF0700001E04000077
:108350003E040000F8B557464E464546DE460C0042
:108360000903E0B5490A460F5F0031431E03DB0FE6
:10837000760A9B46530F3343C84E6500C000E40F96
:10838000D2006D0DA24681467F0D9C469046B742B5
:1083900000D1B9E05B46012673409B46EE1BA34526
:1083A00000D183E0002E63DD002F00D0B1E06346F2
:1083B000134300D123E1731E002B00D0BAE1861ACB
:1083C0006346B04280410125C91A4042091A0B0296
:1083D00000D447E149024B0A98464346002B00D19E
:1083E00089E1404600F0C0FB0300083B1F2B00DD85
:1083F0007CE120223000D21A4146D0409940020050
:108400009E400A439D4200DD6AE15D1B6B1C1F2BF1
:1084100000DD94E1202110003500C91A8E40DA40B9
:108420008840DD40711E8E4111000722284300253F
:1084300006433240002A09D00F233340042B05D0D5
:10844000331DB342B641764289191E000B0200D497
:108450003DE26A1C914B55056D0D9A4200D119E120
:108460008F4AF6080A40570752023743120B9BE027
:10847000002E00D0C5E06E1C7605760D012E00DCC6
:1084800048E16746861ACB1BB042BF417F42B846DF
:108490001F004346FF1A3B00B8461B0200D55FE1B0
:1084A00037439AD100220024002579E0002E00DC19
:1084B000FAE0002F00D18DE0784B9D4267D08023F9
:1084C00067461B041F43BC46382E00DC52E163465E
:1084D00013435A1E93411E18864280414042091898
:1084E0000B0200D4BEE06D4B01359D4200D1D2E0BD
:1084F0006B4A73080A4001210E401E435108D307FE
:1085000007221E43324095E71E00164300D045E780
:1085100040E7624B9D423AD0802367461B041F43CD
:10852000BC46382E00DDEBE01F2E00DC3AE13300C4
:108530006746203BDF403B00202E05D04027BF1B75
:108540006646BE40324390464646721E96413343CD
:10855000DAE0002B00D114E26346134300D168E156
:1085600080234E07C008C9081B030643194208D0E0
:108570006046C008184204D163460100D2085E0775
:108580001643F3009946C900720F444D11434B4600
:10859000DE08424B4F073743CA089D4200D16EE0C8
:1085A00012036D05120B6D0D00211203130B0A0D42
:1085B00012051A433B4B2D0513402B435B00E40788
:1085C0005B082343380019003CBC90469946A246FC
:1085D000AB46F8BD6346134311D0731E002B00D089
:1085E00007E186188642804161444042091801250E
:1085F0000B0237D502257BE73E00614691463500E8
:10860000C5E75C46002D00D0E1E00B000343F3D04A
:10861000731C00D1ACE1214B9F4200D13AE1F343FE
:10862000382B00DD6FE11F2B00DD8CE120250E00D3
:10863000ED1AAE40B0460600AA46DE404546354338
:108640002E005546D940A8406346451EA8415B1AF6
:108650009C463043161AB242924163465242991ADE
:108660003D00B4E607223240002A00D0E4E60B4B7E
:10867000F6084F073743CA089D4200D090E73B00F9
:10868000134300D1A6E180231B031A431203120BEC
:10869000024D89E715000022002785E7FF0700004B
:1086A000FFFF7FFFFFFF0F80002E00D0C7E06B1C95
:1086B0005E05760D012E00DCF0E0C84DAB4200D126
:1086C000B9E085180A00854289416244494251183F
:1086D0000722CE076D082E43490832401D00A9E647
:1086E000BF49ED1A114007223240A3E63200283874
:1086F0008240002686E6300000F036FA203073E62D
:10870000634613435A1E9341C61AB0428041404209
:10871000091A5CE60E00674606431743002D5ED13A
:10872000002E00D0F3E0002F00D11EE15C46614630
:1087300091462CE7A94FBE427BD01E00F1E6100007
:108740001F3DE840202B03D04021CB1A9A4016430E
:10875000731E9E410722064332400021002583E715
:10876000161A6346B2428041591A40420B1A984683
:108770005C4632E61F2E00DDABE02027BB1B9A468D
:1087800063465746BB40994613004F46F3401F438C
:108790003B005746BA40571EBA4113436246F24067
:1087A000891898E62027BB1B9A4663465746BB406C
:1087B000994613004F46F3401F433B005746BA40CB
:1087C000571EBA4113436246F240891A9CE7834B15
:1087D0009F425FD080252D047342294320E7002E5D
:1087E0000CD1002F00D1D0E05C46614691467B4D14
:1087F000CDE67A4FBE421CD01E0065E6002F18D091
:10880000C0084E0706438020C9080003014208D073
:108810006346DC08044204D12100DA46D2085E0730
:108820001643F300994601245346C900720F1143C1
:108830001C406A4DABE61D0000220027B4E6002D67
:1088400059D10B00034300D1D6E6731C00D1B2E02E
:10885000624B9F421ED0F343382B6FDC1F2B00DD91
:1088600097E020250E00ED1AAE40B0460600AA465D
:10887000DE40454635432E005546A840D940451EAA
:10888000A8418C440643B618964292415142614435
:108890003D0025E63D006146914678E60B00034326
:1088A000002D00D055E6002BF5D06346134300D1D0
:1088B0006DE68618864280416144404209180022D4
:1088C0000B0200D4D0E6464B01351940B2E5B14663
:1088D0005DE633006746203BDF403B00202E05D09D
:1088E0004027BF1B6646BE40324390464646721E36
:1088F00096413343EFE5394B9F42CBD080252D0481
:1089000073422943A8E70843411E8841A2E6002F8D
:1089100000D13CE66346861ACF1AB0429B415B42C7
:10892000FB1A98461B024ED5161A6346B242924174
:10893000591A5242891A5C4600227BE501430E0017
:10894000711E8E419FE71D000E00203DEE40B04697
:10895000202B04D04025EB1A994008438146484615
:108960004346411E8841184374E60022002417E65E
:10897000161A6346B2429241591A5242891A3D0070
:1089800025E561469146154D01E68022002412033B
:1089900079E61D000E00203DEE40B046202B04D0AD
:1089A0004025EB1A9940084381464E464346711EC6
:1089B0008E411E4367E7861896429B4161445B42A5
:1089C000C9183D008CE547463743CED007224146C3
:1089D000324049E600273A00E6E5C046FF070000BE
:1089E000FFFF7FFF30B5144D0A034B00120B5B0DE8
:1089F000C90F0024AB4211DD104CA34210DC8024CF
:108A0000640322430E4CE41A1F2C0CDD0D48C31ADC
:108A1000DA4013005C42002900D11C00200030BD68
:108A2000094BCC18FAE7094DE040AC4663449A4044
:108A300013000343EEE7C046FE0300001D040000E0
:108A40003304000013040000FFFFFF7FEDFBFFFF76
:108A500070B500282DD0C317C5185D40C40F28007D
:108A600000F082F8154B1B1A5B055B0D0A2815DD1B
:108A70000B38854000222D032D0B002110002D0303
:108A80000A0D2D0B12052A430D4D1B052A401343D9
:108A90005B00E4075B082343190070BD0200290056
:108AA000153291400A000B21081AC5402D032D0BE9
:108AB000E3E70024002300250022DEE71E04000077
:108AC000FFFF0F804100090E4B1C70B5DBB2460260
:108AD000750AC40F012B14DDE0239B006D07360BD4
:108AE000CB1800210A0D280012051C4D32435B05EE
:108AF0002A405B0813435B00E4075B08234319002B
:108B000070BD002914D1002D1ED0280000F02CF8D3
:108B10000A281CDC0B232A001B1ADA400300153339
:108B20009D400F4B12031B1A5B05160B5B0DD8E71C
:108B3000002D06D0320B802636036D071643094BF5
:108B4000CFE7084B0026CCE700230026C9E7030047
:108B50002A000B3B9A400025E3E7C046FFFF0F8049
:108B600089030000FF0700001C2101231B04984219
:108B700001D3000C10391B0A984201D3000A0839AE
:108B80001B09984201D30009043902A2105C401865
:108B90007047C04604030202010101010000000009
:108BA0000000000030B51C00094B05001B6885B0B3
:108BB000D868084B002A01D1074B1A000292019392
:108BC00000912B002200054900F020F800F01EFE65
:108BD0006400002018B6000087A5000025B600003C
:108BE000084B10B50400002B02D0002100E000BFAC
:108BF000054B1868836A002B00D09847200001F0CD
:108C000029FBC0460000000054B600000EB403B5B6
:108C1000010003AB044804CB0068019300F020F985
:108C200002B008BC03B018476400002070B50026ED
:108C30000C4D0D4C641BA410A64209D1002601F076
:108C40000BFB0A4D0A4C641BA410A64205D170BD53
:108C5000B300EB5898470136EEE7B300EB5898475E
:108C60000136F2E7340200203402002034020020F2
:108C70004402002010B5034B0100186800F06AF8A8
:108C800010BDC0466400002010B5034B01001868F9
:108C900000F016F810BDC04664000020002310B597
:108CA0009A4200D110BDCC5CC4540133F8E70300F4
:108CB0001218934200D1704719700133F9E7000090
:108CC00070B50500002910D00C1F2368002B00DAB6
:108CD000E418280000F0CCFF1D4A1368002B05D1D2
:108CE00063601460280000F0C4FF70BDA34209D97E
:108CF000216860188342F3D118685B6841182160CD
:108D0000EEE713005A68002A01D0A242F9D9196887
:108D10005818A0420BD120680918581819608242CF
:108D2000E0D110685268411819605A60DAE7A04231
:108D300002D90C232B60D5E721686018824203D149
:108D4000106852684118216062605C60CAE7C046E2
:108D50000C120020032370B5CD1C9D43083506007E
:108D60000C2D1ED20C25A9421DD8300000F080FF2A
:108D7000254A14682100002919D1244C2368002BAE
:108D800003D1300000F04EFB20602900300000F0DD
:108D900049FB431C2BD10C233000336000F069FFEA
:108DA00003E0002DDFDA0C233360002070BD0B6878
:108DB0005B1B19D40B2B03D90B60CC18256003E087
:108DC0004B688C420DD11360300000F052FF200040
:108DD00007220B30231D9043C31AE7D05A42E250BA
:108DE000E4E763600C00EFE70C004968C3E7032386
:108DF000C41C9C43A042E1D0211A300000F012FBB9
:108E0000431CDBD1C7E7C0460C1200201012002023
:108E1000936810B5013B9360002B04DA9469A34278
:108E200007DB0A2905D01368581C10601970080068
:108E300010BD00F01FFC0100F9E7F8B506000F00B7
:108E40001400D518AC4201D1002007E021783A0087
:108E50003000FFF7DDFF0134431CF3D1F8BD000003
:108E6000F0B59FB002900F0016000593002805D0C2
:108E700083690493002B01D100F0C8FD7B4B9F4216
:108E80005BD1029B5F68BB891B0762D53B69002BE6
:108E90005FD0002306AC6361203363761033A37682
:108EA00035002B78002B01D0252B5CD1AB1B049314
:108EB0000CD0320039000298FFF7BFFF431C00D1ED
:108EC000C4E06269049B9446634463612B78002B81
:108ED00000D1BBE0012200235242626002A9543259
:108EE00052186E1C2360E360A3601370A365317891
:108EF00005225F4800F09EFE751C002835D12268CF
:108F0000D30604D5532302A95B1820211970130737
:108F100004D5532302A95B182B21197033782A2B0F
:108F20002CD0350000210A20E3682A786E1C303AE4
:108F3000092A64D900292ED026E04E4B9F4202D147
:108F4000029B9F689FE74C4B9F429CD1029BDF682E
:108F500099E73900029800F0E3FB002899D001203E
:108F600040421FB0F0BD01359BE7414B2268C01A5B
:108F700001238340134323602E00B8E7059B191D8E
:108F80001B680591002B01DB099304E05B42E36061
:108F90000223134323602B782E2B0AD16B782A2BC4
:108FA00035D1059B02351A1D1B680592002B2BDB62
:108FB0000793324E29780322300000F03BFE002850
:108FC00006D04023801B8340226801351343236071
:108FD000297806222A486E1C217600F02BFE0028F4
:108FE0003AD0284B002B25D10722059B073393430A
:108FF000083305936369039A9B18636150E7434301
:1090000001219B18350090E701235B42D0E7002344
:109010000A201A000135636029786E1C303909294D
:1090200003D9002BC5D00792C3E74243012352184E
:109030003500F1E705AB00933A00134B210002988D
:1090400000E000BF0390039B0133D3D1BB895B06D3
:1090500000D584E70B9884E705AB00933A000A4BF0
:109060002100029800F080F8ECE7C046ACB60000A2
:1090700058B60000CCB600008CB600005EB600000A
:1090800062B60000000000003B8E0000F7B515003E
:1090900001938A680B6900900C00934200DA130078
:1090A00022002B6043321278002A01D001332B605A
:1090B00023689B0602D52B6802332B6006272368A2
:1090C0001F4027D0230043331B785A1E9341226848
:1090D000920630D42200019943320098089EB0478E
:1090E000431C25D0062320682A68E1680340002538
:1090F000042B03D18D1AEB43DB171D40A3682269B3
:10910000934201DD9B1AED180027BD4220D10020BB
:1091100010E00137E3682A689B1ABB42D2DD2200C7
:109120000123193201990098089EB047431CF0D1E1
:1091300001204042FEBD3020E1184331087021007B
:109140005A1C45310978A218433202331170C1E725
:10915000220001231A3201990098089EB047431C4F
:10916000E6D00137D1E70000F0B589B004920A00DB
:1091700043320593039002920A7E0C000E9B6E2AE6
:1091800000D186E01FD8632A33D008D8002A00D146
:109190008CE0582A4DD0250042352A7030E0642AF0
:1091A00001D0692AF7D1196825680A1D280629D532
:1091B00008681A60002803DA2D23029A40421370CF
:1091C0006B4E0A274FE0732A74D008D86F2A1FD03D
:1091D000702AE0D1202209680A43226003E0752A40
:1091E00016D0782AD7D12200782145321170614EED
:1091F00022E025001A684235111D196013682B7092
:10920000012365E008681A606906D3D500B2D1E78A
:1092100019682568081D186008682E0605D5544E83
:1092200008276F2A1BD00A2719E06D06F7D580B2F0
:10923000F5E745314E4E0A7018682268011D006836
:109240001960150621D5D30702D520231A432260C1
:109250001027002803D1202322689A43226023008C
:10926000002243331A706368A360002B58DB04228A
:10927000216891432160002854D1029D002B5AD0CF
:109280002500337842352B7055E05506DBD580B28A
:10929000D9E71A680D68101D4969186013682E0611
:1092A00001D5196002E06D06FBD519800023029DEF
:1092B00023614FE01A68111D19601568002162686A
:1092C000280000F0B7FC002801D0401B60606368F4
:1092D00023610023029A13703CE023692A00049959
:1092E0000398059DA847431C3ED023689B0715D4CF
:1092F000079BE068984239DA180037E02200012322
:10930000193204990398059EB047431C2CD00135AF
:10931000E368079A9B1AAB42F0DCE9E70025F7E720
:109320000028ADD0029D3900FDF79CFE735C013D25
:109330002B700028F7D1082F09D12368DB0706D549
:1093400063682269934202DC3023013D2B70029B4B
:109350005B1B2361059B07AA00932100049B0398D4
:10936000FFF794FE431CB8D10120404209B0F0BD84
:1093700069B600007AB600000D4B70B51C68050098
:10938000A36B002B0FD11820FFF774FC094BA063CF
:109390000360094B01224360084B83600B238381E8
:1093A0000023026143610022A36B1D615A6170BDFD
:1093B000640000200E33CDAB34126DE6ECDE050008
:1093C000124B10B51C68A36B002B0FD11820FFF7B0
:1093D00051FC0F4BA06303600E4B012243600E4B08
:1093E00083600B238381002302614361A46B0B4ADA
:1093F000206961690A4BFDF771FF01220023801883
:109400005941206161614800400810BD640000209E
:109410000E33CDAB34126DE6ECDE05002D7F954C9E
:109420002DF45158002370B5064C05000800236048
:1094300000F0FAFE431C03D12368002B00D02B6000
:1094400070BDC046C42500200CB430B5164B9DB08D
:109450000C1E1D6808DA8B2301202B6040421DB0D2
:1094600030BC08BC02B01847822302A99B008B8144
:109470000023029008619C4200D0631E8B604B6108
:1094800001235B42CB81209A21AB2800019300F09D
:1094900079FC431C01DA8B232B60002CDFD00023E6
:1094A000029A1370DBE7C046640000200EB400B5DA
:1094B0000B499CB01DAB029006900791049109489E
:1094C000094904CB0591006802A9019300F05AFCF8
:1094D0000023029A13701CB008BC03B01847C046A2
:1094E000FFFFFF7F640000200802FFFF02780B7877
:1094F000002A03D0013001319A42F7D0D01A7047C8
:1095000003000A7801311A700133002AF9D170473B
:109510000023C25C0133002AFBD1581E704730B5CE
:109520000500002A00D130BD0C78013A6B1C2C706C
:109530000131002C05D19A189A42F4D01C700133E5
:10954000FAE71D00EDE70000F0B51F000E0087B040
:109550000590019102920C98347800F0EAFA082202
:1095600000194378751C134036D12D2C36D1B51C0B
:1095700074780126002F62D0102F09D1302C07D12A
:1095800020222B789343582B54D110276C78023526
:109590002D4B3900F31818000393FDF763FD049178
:1095A00001210023494202008C4618002100303975
:1095B00009291AD80C00A74223DD591C09D063469B
:1095C000824206D302D10499A14202DB01237843EF
:1095D00020182C780135E9E72E00BCE72B2C01D0B0
:1095E0001E00C7E7B51C7478FAE721004139192934
:1095F00001D8373CDFE721006139192901D8573CF0
:10960000D9E75A1C08D1059A23331360029B0398AB
:10961000002B09D107B0F0BD002E00D04042029AC5
:10962000002AF7D0002B01D06B1E0193029B019AF8
:109630001A60EFE73024002FAAD10827A8E7302CC2
:109640009ED00A27A4E7C046FFFFFF7F37B513006F
:10965000064A05001068046A002C00D1044C0A0078
:1096600000942900FFF770FF3EBDC0466400002053
:10967000C8000020F8B505000E001400002804D032
:109680008369002B01D100F0C1F9224B9C422DD1FE
:109690006C68A369A360A3891B0731D52369002BDC
:1096A0002ED023682269F7B2981A6369F6B2834212
:1096B00005DC2100280000F03BF9002826D1A36832
:1096C0000130013BA36023685A1C22601F7063694C
:1096D000834204D0A389DB071AD50A2E18D12100B2
:1096E000280000F025F9002812D00FE00A4B9C4218
:1096F00001D1AC68CDE7094B9C42CAD1EC68C8E700
:109700002100280000F00CF80028CAD0012676427B
:109710003000F8BDACB60000CCB600008CB600003E
:10972000364B70B51D6806000C00002D05D0AB69E6
:10973000002B02D1280000F069F9314B9C420FD177
:109740006C680C23E25E93B219072DD4D90611D4AC
:1097500009230120336037331343A381404270BD96
:10976000284B9C4201D1AC68EBE7274B9C42E8D1E7
:10977000EC68E6E75B0713D5616B002908D023008E
:109780004433994202D03000FFF79AFA0023636312
:109790002422A3899343A381002363602369236068
:1097A0000823A2891343A3812369002B0BD1A02195
:1097B0008022A389890092000B40934203D02100AC
:1097C000300000F0E1F90123A289134011D00023F9
:1097D000A36063695B42A361002023698342BED119
:1097E0000C23E25E1306BAD540231343A38101384C
:1097F000B5E7920700D46369A360EDE76400002039
:10980000ACB60000CCB600008CB6000010B5062047
:1098100000F0E0FB012000F01DFD0000F7B58A8993
:1098200005000C00130760D44B68002B04DC0B6CA4
:10983000002B01DC0020FEBDE76A002FFAD00023D8
:109840002E682B6080235B01216A1A4034D0606D42
:10985000A3895B0706D56368C01A636B002B01D030
:10986000236CC01A0200216A00232800E76AB84767
:10987000A189431C06D12B681D2B30D82B4ADA4016
:10988000D3072CD50023636023692360CB0405D55F
:10989000431C02D12B68002B00D16065616B2E60E8
:1098A0000029C7D023004433994202D02800FFF793
:1098B00007FA00206063BEE701232800B847431C75
:1098C000C6D12B68002BC3D01D2B01D0162B01D184
:1098D0002E60AFE74023A2891343A381ABE7402367
:1098E0000B430120A3814042A5E70F69002FA1D0BF
:1098F0000B680F60DB1B01930023920700D14B69BB
:10990000A360019B002B00DC94E7019B3A00216AD5
:109910002800A66AB047002803DC4023A28913432D
:10992000DFE7019B3F181B1A0193EAE70100402083
:109930000B6970B505000C00002B01D1002070BD33
:10994000002804D08369002B01D100F05FF80B4B95
:109950009C4209D16C680C22A35E002BEED0210042
:109960002800FFF75BFFEAE7054B9C4201D1AC689A
:10997000F1E7044B9C42EED1EC68ECE7ACB600009A
:10998000CCB600008CB60000002310B504000360C4
:109990004360836081814366C28103614361836167
:1099A000190008225C30FFF782F9054B24626362DC
:1099B000044BA362044BE362044B236310BDC04617
:1099C00015A000003DA0000075A00000A1A00000AF
:1099D00010B5024900F08CF810BDC0463199000066
:1099E00070B568254A1E55430E0029007431FFF7F3
:1099F000B1F9041E08D000212A00016046600C3035
:109A0000A0606832FFF753F9200070BD836913B579
:109A10000400002B28D18364C3640365134B144AEC
:109A20001B6882620193984201D101238361200067
:109A300000F020F86060200000F01CF8A06020001A
:109A400000F018F80022E06004216068FFF79CFF36
:109A500001220921A068FFF797FF02221221E06886
:109A6000FFF792FF0123A36113BDC04654B6000067
:109A7000D1990000F8B51C4B07001E68B369002B94
:109A800002D13000FFF7C2FF4836B4687368013B6B
:109A900004D53368002B07D03668F6E70C22A55EA4
:109AA000002D0DD06834F2E704213800FFF798FF4D
:109AB00030600028F0D10C2304003B602000F8BD8A
:109AC00020000A4B656625606560A560E36025613E
:109AD0006561A561082229005C30FFF7E8F865633D
:109AE000A563A564E564E9E754B600000100FFFF43
:109AF000F7B504000700002601914834002C01D17D
:109B00003000FEBD6368A5680093009B013B009395
:109B100001D52468F2E7AB89012B08D90E22AB5E90
:109B2000013304D029003800019B9847064368356B
:109B3000EBE7EC300068704770B50E001D000E2397
:109B4000C95E96B01400002907DA00232B60B389A0
:109B50001B0611D48023DB000FE06A4600F0D8FA20
:109B60000028F2DBF022019B12021340054A9B18E9
:109B70005A4253412B60EDE740230020236016B08A
:109B800070BDC04600E0FFFFF7B502268B890500D7
:109B90000C00334206D023004733236023610123A6
:109BA0006361F7BD01AB6A46FFF7C6FF0099070086
:109BB0002800FFF7CFF8002808D10C22A35E9A05F1
:109BC000EFD4032293431E43A681E4E70F4BAB621D
:109BD0008023A28920601343A381009B20616361DD
:109BE000019B002B0DD00E23E15E280000F0A2FAAD
:109BF000002806D00322A38993431A0001231343AC
:109C0000A381A0893843A081CBE7C046D199000049
:109C100082B0002900D101A9101E06D0002B06D069
:109C200013780B601078431E984102B070470220F1
:109C30004042FAE7C9B28218904201D10020704731
:109C400003788B42FBD00130F6E710B5884202D989
:109C50008B18984203D3002307E08B5C8354013AAE
:109C6000FBD210BDCC5CC45401339A42FAD1F8E760
:109C700070477047F8B507000D001600002905D1A0
:109C80001100FFF767F804002000F8BD002A03D197
:109C9000FFF716F83400F7E700F072FA2C00B04234
:109CA000F2D231003800FFF755F8041EECD029003D
:109CB0003200FEF7F3FF29003800FFF701F8E3E771
:109CC000F0B58E6885B007000C00039201939E42A8
:109CD0003CD890238A89DB001A4234D003250969D5
:109CE00023685B1A0293636902985D43EB0F5D1969
:109CF000019B6D1001331B18AB4200D91D005305A9
:109D000032D529003800FFF725F8061E09D10C23AB
:109D10003B6040230120A28940421343A38105B048
:109D2000F0BD029A2169FEF7B9FFA389144A1A40CF
:109D300080231343A381029B2661F6182660656188
:109D4000019EED1AA560019B9E4200D9019E320042
:109D500003992068FFF779FFA36800209B1BA3608D
:109D600023689E192660DAE72A003800FFF782FF91
:109D7000061EE0D121693800FEF7A2FFC7E7C04602
:109D80007FFBFFFFF0B59FB0029005938B890F001A
:109D900016001B0611D50B69002B0ED14021FEF7D2
:109DA000D9FF38603861002805D10C23029A0138A8
:109DB00013601FB0F0BD40237B61002306AC6361DC
:109DC000203363761033A37635002B78002B01D037
:109DD000252B46D1AB1B04930CD0320039000298DE
:109DE000FFF76EFF431C00D1AEE06269049B94460E
:109DF000634463612B78002B00D1A5E0012200238E
:109E00005242626002A9543252186E1C2360E36011
:109E1000A3601370A365317805225448FFF70AFF49
:109E2000751C00281FD12268D30604D5532302A92C
:109E30005B1820211970130704D5532302A95B185E
:109E40002B21197033782A2B16D0350000210A20D7
:109E5000E3682A786E1C303A092A4ED9002918D0B6
:109E600010E00135B1E7414B2268C01A012383405D
:109E7000134323602E00CEE7059B191D1B68059137
:109E8000002B01DB099304E05B42E36002231343F0
:109E900023602B782E2B0AD16B782A2B35D1059B8A
:109EA00002351A1D1B680592002B2BDB0793304EE1
:109EB000297803223000FFF7BDFE002806D040239A
:109EC000801B8340226801351343236029780622D2
:109ED00028486E1C2176FFF7ADFE00283CD0264BAB
:109EE000002B25D10722059B0733934308330593A5
:109EF0006369039A9B18636166E7434301219B18DA
:109F00003500A6E701235B42D0E700230A201A00B0
:109F10000135636029786E1C3039092903D9002B7B
:109F2000C5D00792C3E74243012352183500F1E739
:109F300005AB00933A00114B2100029800E000BFEE
:109F40000390039B0133D3D1BB890B985B0600D4EC
:109F50002FE7012040422CE705AB00933A00074B66
:109F600021000298FFF700F9EAE7C04658B6000062
:109F70005EB6000062B6000000000000C19C000058
:109F800070B504000D001F2904D9162303600120B9
:109F9000404270BD436C002B04D08A009B181A68A5
:109FA000002A08D1200000F031F82A00010020002A
:109FB00000F01AF8EDE70020012AEAD0511C03D185
:109FC000162301302360E4E7002428001C6090473A
:109FD0002000DEE710B5034B01001868FFF7D0FF43
:109FE00010BDC04664000020002370B5064C05007B
:109FF00008001100236000F0FFF8431C03D1236820
:10A00000002B00D02B6070BDC425002010B500F0DF
:10A01000E3F810BD70B50C000E25495F00F0B8F8EC
:10A02000002803DB636D1B18636570BDA389024ABA
:10A030001340A381F9E7C046FFEFFFFFF8B51F000B
:10A040008B8905000C001600DB0505D50E23C95EC3
:10A050000022022300F080F8A389054A280013405B
:10A06000A38132000E23E15E3B0000F02BF8F8BD27
:10A07000FFEFFFFF70B50C000E25495F00F06CF894
:10A08000A389421C03D1054A1340A38170BD8022DD
:10A0900052011343A3816065F8E7C046FFEFFFFF5D
:10A0A00010B50E23C95E00F021F810BD0B1E04D0C0
:10A0B000FF2A04D98A2303608B3B180070470A707B
:10A0C0000123FAE770B50500080011000022064CD4
:10A0D00022601A0000F0B6F8431C03D12368002B5D
:10A0E00000D02B6070BDC046C4250020002370B591
:10A0F000064C05000800236000F05EF8431C03D105
:10A100002368002B00D02B6070BDC046C425002002
:10A11000002370B5064C050008001100236000F014
:10A1200053F8431C03D12368002B00D02B6070BD73
:10A13000C4250020002370B5064C050008002360EC
:10A1400000F052F8431C03D12368002B00D02B6091
:10A1500070BDC046C425002070B505000800110080
:10A160000022064C22601A0000F04EF8431C03D176
:10A170002368002B00D02B6070BDC046C425002092
:10A180000B1F1B68181F002B01DA0B58C0187047F3
:10A1900070B50500080011000022064C22601A006C
:10A1A00000F03AF8431C03D12368002B00D02B6049
:10A1B00070BDC046C425002058220120014B4042FA
:10A1C0001A607047C425002058220120014B4042EC
:10A1D0001A607047C425002058220120014B4042DC
:10A1E0001A607047C42500205822024B00201A60D4
:10A1F0007047C046C425002058220120014B404230
:10A200001A607047C425002058220120014B4042AB
:10A210001A607047C425002058220120014B40429B
:10A220001A607047C4250020044A1368002B00D12F
:10A23000034B1818106018007047C0461412002015
:10A24000C825002058220120014B40421A60704767
:10A25000C4250020FEE7C046F8B5C046F8BC08BCDF
:10A260009E467047F8B5C046F8BC08BC9E4670478D
:10A2700054050000640500007E050000FC05000098
:10A28000340600006A060000A2060000C8060000AE
:10A2900004070000460700009C070000E0070000DC
:10A2A0004C08000094080000BA080000F208000002
:10A2B000380900005E0900008C090000BE0900009A
:10A2C000F60900007A0A0000460B0000BC0B0000F3
:10A2D000280C0000700C0000900C0000B20C000074
:10A2E0008C0D0000D20D0000540500005405000044
:10A2F000540500004A0E0000B20E0000340F0000AA
:10A300007A0F0000C20F000040100000BE100000D5
:10A31000061100004C11000082110000C81100005D
:10A320000E12000056120000AA12000008130000CE
:10A3300046130000B0130000E61300002E140000C6
:10A3400076140000BE140000F81400004015000050
:10A350008815000054050000540500005405000055
:10A36000F0150000261600005C160000881600009C
:10A37000BE160000F416000054050000540500004D
:10A3800054050000540500002A1700006C17000057
:10A390005405000054050000B21700000218000028
:10A3A0002818000054050000540500005405000062
:10A3B0005618000086180000B6180000EC180000BF
:10A3C000161900004C190000761900009E190000B3
:10A3D000C6190000F6190000261A0000501A0000E5
:10A3E0007A1A0000AA1A0000EC1A000054050000B6
:10A3F00054050000540500005405000054050000F9
:10A400001C1B0000481B0000741B0000A01B000068
:10A41000CC1B0000021C0000381C00006E1C000059
:10A42000A41C0000D01C0000FC1C0000321D000019
:10A4300054050000540500005405000054050000B8
:10A4400054050000540500005405000054050000A8
:10A450005405000054050000540500005405000098
:10A4600054050000540500005E1D00008A1D000018
:10A4700066616C73650074727565006C6973742035
:10A480006F66202564206974656D73006F626A656C
:10A490006374206F6620636C6173733A20256400D7
:10A4A000537461636B20756E646572666C6F7700C0
:10A4B0000700000003000000FAA40000651E000071
:10A4C00002A50000691E00000BA50000611E00002F
:10A4D00014A500006D1E0000000000000100000037
:10A4E0000200000003000000040000000A00000059
:10A4F0006D6963726F3A62697400686173546F6E5C
:10A500006500706C6179546F6E65006861735365A6
:10A5100072766F00736574536572766F00496E735F
:10A52000756666696369656E74206D656D6F7279B5
:10A5300020666F72204D6963726F426C6F636B733C
:10A54000206F626A656374206865617000496E738C
:10A55000756666696369656E74206D656D6F727985
:10A5600020666F72204D6963726F426C6F636B730C
:10A5700020737461636B000D0A564D2050616E6943
:10A58000633A2025730D0A006D69736300000000B3
:10A59000A0A5000075230000A9A500002D23000040
:10A5A000686578546F496E740073696E000000002E
:10A5B000FCA50000E123000004A60000E523000044
:10A5C0000EA600000324000017A600000D240000C2
:10A5D00022A60000172400002EA60000212400005F
:10A5E0003FA600002B24000055A60000EF2300002A
:10A5F0006EA60000F92300006E6574006861735751
:10A6000069466900737461727457694669007374AE
:10A610006F7057694669007769666953746174752C
:10A6200073006D7949504164647265737300746896
:10A63000696E674465736372697074696F6E0063F5
:10A640006C6561725468696E6744657363726970A2
:10A6500074696F6E00617070656E64546F546869E0
:10A660006E674465736372697074696F6E006170C0
:10A6700070656E64546F5468696E6750726F706570
:10A68000727479001A1B1C03040607090A171819AB
:10A6900003040607090A171819000000000008083B
:10A6A0000800080A4A4000000A5FEA5FEA0ED92E55
:10A6B000D36E19324489330C924C924D0808000035
:10A6C0000004880808040804848488000A448A4036
:10A6D00000048EC480000000048800000EC000004A
:10A6E0000000080001224488100C9252524C048C45
:10A6F00084848E1C824C901E1EC244924C06CA5208
:10A700005FE21FF01EC13E02448ED12E1FE244883C
:10A71000100ED12ED12E0ED12EC4880008000800B4
:10A7200000048004880244880482000EC00EC00821
:10A73000048244880ED126C0040ED135B36C0C922D
:10A740005ED2521C925C925C0ED010100E1C925283
:10A75000525C1ED01C901E1ED01C90100ED0137187
:10A760002E12525ED2521C8808081C1FE242524C24
:10A770001254981492101010101E113B75B1311123
:10A780003935B3710C9252524C1C925C90100C9261
:10A79000524C861C925C92510ED00C825C1FE48459
:10A7A0008484125252524C1131312A44113135BB3A
:10A7B0007112524C9252112A4484841EC488101E75
:10A7C0000EC808080E10080482410EC242424E0410
:10A7D0008A400000000000001F0804800000000EF6
:10A7E000D2524F10101C925C000ED0100E02424E3E
:10A7F000D24E0C925C900E06C81C88080ED24EC237
:10A800004C10101C92520800080808024002424CEA
:10A8100010149814920808080806001B75B131003E
:10A820001C925252000C92524C001C925C90000EF2
:10A83000D24EC2000ED010100006C8049808080EB0
:10A84000C807001252524F0011312A44001131350D
:10A85000BB00124C8C9200112A4498001EC4881E22
:10A8600006C48C8486080808080818080C88180094
:10A87000000C8360000000000100000002000000E6
:10A8800003000000040000000500000006000000B6
:10A890000700000008000000090000000A00000096
:10A8A0000B0000000C0000000D0000000E00000076
:10A8B0000F00000010000000120000001400000053
:10A8C00016000000180000001A0000001C00000024
:10A8D0001E000000200000002300000026000000F1
:10A8E000290000002C0000002F00000032000000B2
:10A8F000360000003A0000003E0000004200000068
:10A90000460000004B000000500000005500000011
:10A910005A00000061000000680000006F000000A5
:10A92000760000007D000000840000008B00000025
:10A930009200000099000000A0000000A7000000A5
:10A94000AE000000B5000000BC000000C300000025
:10A95000CA000000D1000000D8000000DF000000A5
:10A96000E6000000ED000000F4000000FB00000025
:10A97000FF000000C4A9000051240000CFA900007E
:10A9800021290000D9A9000031260000E6A9000015
:10A9900051260000EDA90000A1260000F6A9000044
:10A9A000F126000002AA00004D29000013AA0000B1
:10A9B0006528000020AA0000312800006469737037
:10A9C0006C6179006C696768744C6576656C006DC4
:10A9D00062446973706C6179006D62446973706C74
:10A9E00061794F6666006D62506C6F74006D6255E0
:10A9F0006E706C6F74006D62447261775368617041
:10AA000065006D625368617065466F724C65747461
:10AA10006572006E656F506978656C53656E640091
:10AA20006E656F506978656C53657450696E004E41
:10AA30006F7420656E6F75676820726F6F6D20652B
:10AA400076656E20616674657220636F6D706163F8
:10AA500074696F6E00436F6D706163746564204646
:10AA60006C61736820636F64652073746F72650A2C
:10AA700025642062797465732075736564202825C8
:10AA800064252529206F66202564004261642072B8
:10AA900065636F726420666F756E64206475726999
:10AAA0006E6720696E697469616C697A6174696F37
:10AAB0006E002564202564202564202825642077E5
:10AAC0006F72647329002564207265636F7264730A
:10AAD0002C20256420776F7264732C206D61784977
:10AAE000442025642C20636F6D70616374696F6E00
:10AAF000206379636C657320256400526573746FFD
:10AB000072656420256420736372697074730053E6
:10AB100074617274656400726164696F00000000A2
:10AB2000AEAB000051330000BBAB0000BD350000F0
:10AB3000CBAB000061350000D9AB00003D37000011
:10AB4000E4AB000069330000F4AB0000DD3300002B
:10AB500008AC00007933000017AC00001D3900007C
:10AB600023AC00009D3800002CAC000041380000F0
:10AB700037AC00008937000042AC0000C537000048
:10AB80004BAC0000F937000054AC00008D330000DE
:10AB90006E756D626572006E6F6E65006F746865CC
:10ABA00072007061697200737472696E6700646923
:10ABB0007361626C65526164696F006D6573736186
:10ABC00067655265636569766564007061636B658E
:10ABD0007452656365697665007061636B65745373
:10ABE000656E64007265636569766564496E746557
:10ABF0006765720072656365697665644D65737338
:10AC0000616765547970650072656365697665642E
:10AC1000537472696E670073656E64496E7465671C
:10AC200065720073656E64506169720073656E646D
:10AC3000537472696E67007365744368616E6E6504
:10AC40006C0073657447726F757000736574506F34
:10AC5000776572007369676E616C537472656E67B5
:10AC60007468000000000000963007772C610EEE3B
:10AC7000BA51099919C46D078FF46A7035A563E953
:10AC8000A395649E3288DB0EA4B8DC791EE9D5E07A
:10AC900088D9D2972B4CB609BD7CB17E072DB8E779
:10ACA000911DBF906410B71DF220B06A4871B9F3CE
:10ACB000DE41BE847DD4DA1AEBE4DD6D51B5D4F407
:10ACC000C785D38356986C13C0A86B647AF962FD6C
:10ACD000ECC9658A4F5C0114D96C0663633D0FFAB9
:10ACE000F50D088DC8206E3B5E10694CE44160D5BF
:10ACF000727167A2D1E4033C47D4044BFD850DD2A9
:10AD00006BB50AA5FAA8B5356C98B242D6C9BBDBBB
:10AD100040F9BCACE36CD832755CDF45CF0DD6DCB6
:10AD2000593DD1ABAC30D9263A00DE518051D7C85D
:10AD30001661D0BFB5F4B42123C4B3569995BACFE8
:10AD40000FA5BDB89EB802280888055FB2D90CC609
:10AD500024E90BB1877C6F2F114C6858AB1D61C182
:10AD60003D2D66B69041DC760671DB01BC20D298A1
:10AD70002A10D5EF8985B1711FB5B606A5E4BF9F2E
:10AD800033D4B8E8A2C9077834F9000F8EA8099621
:10AD900018980EE1BB0D6A7F2D3D6D08976C64918C
:10ADA000015C63E6F4516B6B62616C1CD8306585A5
:10ADB0004E0062F2ED95066C7BA5011BC1F4088282
:10ADC00057C40FF5C6D9B06550E9B712EAB8BE8BC3
:10ADD0007C88B9FCDF1DDD62492DDA15F37CD38C4C
:10ADE000654CD4FB5861B24DCE51B53A7400BCA34A
:10ADF000E230BBD441A5DF4AD795D83D6DC4D1A47C
:10AE0000FBF4D6D36AE96943FCD96E34468867AD52
:10AE1000D0B860DA732D0444E51D03335F4C0AAAF1
:10AE2000C97C0DDD3C710550AA41022710100BBEF4
:10AE300086200CC925B56857B3856F2009D466B93B
:10AE40009FE461CE0EF9DE5E98C9D9292298D0B070
:10AE5000B4A8D7C7173DB359810DB42E3B5CBDB71D
:10AE6000AD6CBAC02083B8EDB6B3BF9A0CE2B6039E
:10AE70009AD2B1743947D5EAAF77D29D1526DB0453
:10AE80008316DC73120B63E3843B64943E6A6D0D9E
:10AE9000A85A6A7A0BCF0EE49DFF099327AE000AE9
:10AEA000B19E077D44930FF0D2A3088768F2011E7C
:10AEB000FEC206695D5762F7CB67658071366C1913
:10AEC000E7066B6E761BD4FEE02BD3895A7ADA1034
:10AED000CC4ADD676FDFB9F9F9EFBE8E43BEB71715
:10AEE000D58EB060E8A3D6D67E93D1A1C4C2D8389F
:10AEF00052F2DF4FF167BBD16757BCA6DD06B53F05
:10AF00004B36B248DA2B0DD84C1B0AAFF64A033643
:10AF1000607A0441C3EF60DF55DF67A8EF8E6E31C2
:10AF200079BE69468CB361CB1A8366BCA0D26F250B
:10AF300036E2685295770CCC03470BBBB916022258
:10AF40002F260555BE3BBAC5280BBDB2925AB42B6D
:10AF5000046AB35CA7FFD7C231CFD0B58B9ED92C82
:10AF60001DAEDE5BB0C2649B26F263EC9CA36A75E7
:10AF70000A936D02A906099C3F360EEB856707729E
:10AF800013570005824ABF95147AB8E2AE2BB17B05
:10AF9000381BB60C9B8ED2920DBED5E5B7EFDC7C8C
:10AFA00021DFDB0BD4D2D38642E2D4F1F8B3DD68E3
:10AFB0006E83DA1FCD16BE815B26B9F6E177B06FDE
:10AFC0007747B718E65A0888706A0FFFCA3B0666CB
:10AFD0005C0B0111FF9E658F69AE62F8D3FF6B6158
:10AFE00045CF6C1678E20AA0EED20DD75483044EFA
:10AFF000C2B30339612667A7F71660D04D47694988
:10B00000DB776E3E4A6AD1AEDC5AD6D9660BDF409A
:10B01000F03BD83753AEBCA9C59EBBDE7FCFB2474D
:10B02000E9FFB5301CF2BDBD8AC2BACA3093B35332
:10B03000A6A3B4240536D0BA9306D7CD2957DE543B
:10B04000BF67D9232E7A66B3B84A61C4021B685D14
:10B05000942B6F2A37BE0BB4A18E0CC31BDF055A8D
:10B060008DEF022D416C6C207461736B73207374CF
:10B070006F707065640076303639002025732025A6
:10B0800073004D656D6F727920636C6561726564E4
:10B09000004E6F2066726565207461736B20656E6B
:10B0A0007472696573000000E8B000008147000019
:10B0B000F4B00000E94A0000FAB00000F94A0000CC
:10B0C00000B10000094B000006B10000B5470000C8
:10B0D00010B10000194B000018B10000F548000045
:10B0E00073656E736F72730074656D7065726174F1
:10B0F0007572650074696C74580074696C745900D9
:10B1000074696C745A00746F756368526561640089
:10B1100069326352656164006932635772697465AC
:10B120000000000098B100009D4B0000A6B1000097
:10B13000A14B0000AFB10000AD4B0000B9B1000061
:10B14000B14B0000C2B10000B54B0000C7B1000018
:10B15000B94B0000CCB10000BD4B0000D8B10000DD
:10B16000C14B0000DFB10000C54B0000E8B100009A
:10B17000C94B0000EDB10000CD4B0000F8B100005C
:10B18000D14B000002B20000A54B00000CB2000041
:10B19000A94B000074667400656E61626C65446959
:10B1A00073706C61790067657457696474680067CF
:10B1B000657448656967687400736574506978657B
:10B1C0006C006C696E65007265637400726F756EF9
:10B1D0006465645265637400636972636C650074CE
:10B1E0007269616E676C650074657874007466746A
:10B1F000546F756368656400746674546F75636832
:10B200005800746674546F7563685900746674549A
:10B210006F75636850726573737572650057656CFE
:10B22000636F6D6520746F204D6963726F426C6F40
:10B23000636B732100705F73706920213D204E5550
:10B240004C4C002F686F6D652F62726F6D61676F78
:10B2500073612F2E706C6174666F726D696F2F70E1
:10B2600061636B616765732F6672616D65776F727D
:10B270006B2D61726475696E6F6E6F726469636E57
:10B280007266352F6C69627261726965732F5350F3
:10B29000492F5350492E63707000535049436C61DD
:10B2A00073733A3A535049436C617373284E524654
:10B2B0005F5350495F547970652A2C2075696E740C
:10B2C000385F742C2075696E74385F742C20756932
:10B2D0006E74385F74290000000000000000000058
:10B2E000D94D0000954D0000BB4D0000C54D00003C
:10B2F000CF4D0000B94D0000030000000200000027
:10B300000100000004000000050000001100000022
:10B310000C0000000B000000120000000A000000FA
:10B32000060000001A0000001400000017000000D2
:10B33000160000001500000010000000FFFFFFFFD6
:10B34000FFFFFFFF000000001E00000019000000CA
:10B3500018000000070000000800000009000000BD
:10B360000D0000000E0000000F0000001C00000097
:10B370001B0000001D000000130000000000000082
:10B380000000000089520000B95900000953000074
:10B390001D53000013530000855200007952000035
:10B3A00029530000A5520000755200000000000063
:10B3B000000000000000304300000000000030C327
:10B3C000FB21F93FFB2109407CD91240FB211940A8
:10B3D0007A6A1F407CD92240BBFD2540FB212940D1
:10B3E0003A462C407A6A2F405C4731407CD9324043
:10B3F0009C6B3440BBFD3540DB8F3740FB2139402F
:10B400001BB43A403A463C405AD83D407A6A3F40E5
:10B410004C7E40405C4741406C1042407CD94240E9
:10B420008CA243409C6B4440AC344540BBFD45403E
:10B43000CBC64640DB8F4740EB584840FB21494094
:10B4400083F9A200444E6E00FC291500D157270055
:10B45000DD34F50062DBC0003C999500419043006B
:10B460006351FE00BBDEAB00B761C5003A6E24003D
:10B47000D24D42004906E00009EA2E001C92D1009C
:10B48000EB1DFE0029B11C00E83EA700F535820047
:10B4900044BB2E009CE98400B4267000417E5F000E
:10B4A000D6913900538339009CF439008B5F8400B6
:10B4B00028F9BD00F81F3B00DEFF97000F9805003C
:10B4C000112FEF000A5A8B006D1F6D00CF7E3600E2
:10B4D00009CB2700464FB7009E663F002DEA5F006C
:10B4E000BA277500E5EBC7003D7BF100F73907008F
:10B4F00092528A00FB6BEA001FB15F00085D8D006D
:10B50000300356007BFC4600F0AB6B0020BCCF0044
:10B5100036F49A00E3A91D005E619100081BE60065
:10B5200085996500A0145F008D40680080D8FF00F9
:10B5300027734D0006063100CA561500C9A87300CE
:10B540007BE260006B8CC00000000040FB21F93FF3
:10B55000000000002D44743E000000809846F83C36
:10B560000000006051CC783B00000080831BF03964
:10B570000000004020257A38000000802282E33657
:10B58000000000001DF36935020000000300000008
:10B59000040000000600000028740000D2730000C0
:10B5A000D273000000750000CE730000CE7300005F
:10B5B000F674000000750000CE730000F674000001
:10B5C000CE730000007500000475000004750000D3
:10B5D000047500000C750000288000002A7F000020
:10B5E0002A7F000048820000247F0000247F0000A2
:10B5F0003082000048820000247F0000308200007A
:10B60000247F0000488200003E8200003E8200004D
:10B610003E8200004C8200002C2066756E637469C7
:10B620006F6E3A2000617373657274696F6E2022C9
:10B63000257322206661696C65643A2066696C65D1
:10B6400020222573222C206C696E652025642573C9
:10B6500025730A0068000020232D302B2000686C21
:10B660004C00656667454647003031323334353625
:10B67000373839414243444546003031323334355E
:10B680003637383961626364656600000000000087
:10B6900000000000000000000000000000000000AA
:10B6A000000000000000000000000000000000009A
:10B6B000000000000000000000000000000000008A
:10B6C000000000000000000000000000000000007A
:10B6D000000000000000000000000000000000006A
:10B6E0000000000000000000000000004300504F78
:10B6F000534958002E000020202020202020202008
:10B700002828282828202020202020202020202011
:10B710002020202020202088101010101010101041
:10B720001010101010101004040404040404040485
:10B73000041010101010101041414141414101010D
:10B7400001010101010101010101010101010101E9
:10B7500001011010101010104242424242420202F7
:10B7600002020202020202020202020202020202B9
:10B770000202101010102000000000000000000065
:10B7800000000000000000000000000000000000B9
:10B7900000000000000000000000000000000000A9
:10B7A0000000000000000000000000000000000099
:10B7B0000000000000000000000000000000000089
:10B7C0000000000000000000000000000000000079
:10B7D0000000000000000000000000000000000069
:10B7E0000000000000000000000000000000000059
:0CB7F0000000000000000000000000004D
:08B7FC000C49FF7F0100000071
:10B80400FFFFFFFF400600001800000019FCFFFFC7
:10B81400FFFFFFFFFF000000020000000300000024
:10B82400FFFFFFFF00000000010000000000020015
:10B8340001000000FFFFFFFF000000000200000005
:10B844000000040002000000FFFFFFFF00000000F2
:10B854000300000000000800030000000A000000CC
:10B86400080000006800002000000000ACB60000E2
:10B87400CCB600008CB60000000000000000000000
:10B8840000000000000000000000000000000000B4
:10B8940000000000000000000000000000000000A4
:10B8A4000000000000000000000000000000000094
:10B8B4000000000000000000000000000000000084
:10B8C4000000000000000000430000000000000031
:10B8D4000000000000000000000000000000000064
:10B8E4000000000000000000430000000000000011
:10B8F4000000000000000000000000000000000044
:10B9040000000000000000004300000000000000F0
:10B914000000000000000000000000000000000023
:10B9240000000000000000004300000000000000D0
:10B934000000000000000000000000000000000003
:10B9440000000000000000004300000000000000B0
:10B9540000000000000000000000000000000000E3
:10B964000000000000000000430000000000000090
:10B9740000000000000000000000000000000000C3
:10B984000000000000000000430000000000000070
:10B9940000000000000000000000000000000000A3
:10B9A4000000000000000000ADA00000119C000099
:10B9B40000000000F6B60000F4B6000087A5000001
:10B9C40087A5000087A5000087A5000087A50000C3
:10B9D40087A5000087A5000087A5000087A50000B3
:10B9E400FFFFFFFFFFFFFFFFFFFFFFFFFFFF000061
:10B9F40001004153434949000000000000000000D9
:10BA04000000000000000000000000000000000032
:10BA140000004153434949000000000000000000B9
:10BA24000000000000000000000000000000000012
:10BA340000000000E9000000654D0000AD5000006A
:08BA4400D5550000C10000000F
:04000003000051495F
:00000001FF
